:100000006BC3000086C3000084C3000082C30000ED
:1000100080C300007EC300007CC300007AC30000E0
:1000200078C3000076C300000C94442F0C94103069
:100030000C942C2A6EC300006CC300006AC300003D
:1000400068C3000066C3000064C3000062C3000010
:1000500060C300000C94A32A5CC300005AC30000D4
:1000600058C3000056C3000054C3000052C3000030
:1000700050C300004EC300004CC300004AC3000040
:1000800048C3000046C3000044C3000042C3000050
:1000900040C300003EC300003CC300003AC3000060
:1000A00038C3000036C3000034C30000040005005C
:1000B0000600070008001E001F002000210022008B
:1000C000230024002500260027001E0F0500047FC2
:1000D0003F1F643214643214783C1E1E140A052239
:1000E00023252628292A2C2D2F3032333536383A2D
:1000F0003B3D3E4042434547494A4C4E5051535583
:1001000057595A5C5E6062646668696B6D6F7173A3
:100110007577797B7D7F81838587898A8C8E9092A4
:100120009496989A9C9E9FA1A3A5A7A8AAACAEAFAF
:10013000B1B3B4B6B8B9BBBCBEBFC1C2C3C5C6C7F4
:10014000C9CACBCCCDCED0D1D2D2D3D4D5D6D7D7A5
:10015000D8D9D9DADADBDBDBDCDCDCDCDCDDDDDDED
:10016000DDDCDCDCDCDCDBDBDBDADAD9D9D8D7D7E9
:10017000D6D5D4D3D2D2D1D0CECDCCCBCAC9C7C696
:10018000C5C3C2C1BFBEBCBBB9B8B6B4B3B1AFAED4
:10019000ACAAA8A7A5A3A19F9E9C9A98969492907A
:1001A0008E8C8A89878583817F7D7B797775737152
:1001B0006F6D6B6968666462605E5C5A595755532F
:1001C00051504E4C4A4947454342403E3D3B3A38E8
:1001D00036353332302F2D2C2A292826252322FF8D
:1001E000AA7F554000010101010101010101020244
:1001F00002020202020202030303030303030304D5
:10020000040404040404050505050506060606069F
:10021000070707070708080808090909090A0A0A59
:100220000B0B0B0C0C0C0D0D0D0E0E0E0F0F0F10FB
:100230001011111112121313141415151616171785
:10024000181819191A1A1B1B1C1D1D1E1E1F2020F1
:10025000212222232424252626272829292A2B2C3B
:100260002D2D2E2F30313232333435363738393A5E
:100270003B3C3D3E3F404142434445464748494A56
:100280004C4D4E4F50515354555658595A5B5D5E24
:100290005F616264656668696B6C6D6F70727375BF
:1002A00077787A7B7D7E8082838587888A8C8E8F23
:1002B00091939596989A9C9EA0A2A3A5A7A9ABAD51
:1002C000AFB1B3B5B7BABCBEC0C2C4C6C9CBCDCF3F
:1002D000D1D4D6D8DBDDDFE2E4E7E9EBEEF0F3F5ED
:1002E000F8FAFDFFFD377A585A000004E6D6B44606
:1002F0000200210116000000742FE5A3E003CF01E6
:100300001D5D003D8889C65436C3174FE4F609DCED
:100310009AD594C1FE25E1FB5EB449F901893E23DB
:10032000D12FC383789039A003F752A274A0385F0D
:100330000F24739956423F11C8A112FCD0ED203B07
:1003400080AECCCD19F6E0122EC6877B8BFB4941DF
:1003500040804A064B3C8FCA706099A3F2E1473750
:1003600009B590880F6CF36F58705455E947D32A3C
:1003700011E154EBA1355EE541339F1C750B9E8462
:100380001E0294AA40445A6F81D8347E406E2B9945
:100390002F3089BD6726856B37A60ADE80DF71871F
:1003A00097D9781837858077830DF3B2681ACE26EF
:1003B000AA821E107830A96A2674BBD6AA1F083DEF
:1003C0005C89D59D078D10B432653071F6B5CCDBF4
:1003D000AC15DD110C23DB9990F5F9D51B35C09CCC
:1003E000EB710136B2D07940C2D397C96C7CE0ABD7
:1003F000CD1E59E265EB82EA45BE565367A408BCA0
:100400007944406EFFBBA4B846769390E07C646963
:10041000CCE9095CA6872871EBACE1806151B6009C
:1004200000000000E15F54D90FD3CAB90001B9023E
:10043000D00700001C6A4BA7B1C467FB0200000094
:100440000004595A00000000000000002A2B280078
:100450000000000000000000000000000000002973
:10046000000000002C1E3420212224342627252EB3
:10047000362D3738271E1F202122232425263333EB
:10048000362E37381F0405060708090A0B0C0D0E17
:100490000F101112131415161718191A1B1C1D2FE3
:1004A0003130232D350405060708090A0B0C0D0E03
:1004B0000F101112131415161718191A1B1C1D2FC3
:1004C0003130354C0000000000000000000000004A
:1004D000000000000000000000000000000000001C
:1004E00000000000000000007E0F00D4FFFFFFC7E7
:1004F000000000781C037600690061006C003A007F
:10050000660036003400630032006200330063008E
:10051000000016036D0069006E0069004D00410087
:10052000430052004F00350000001E036C006500C0
:10053000610066006300750074007400650072005D
:100540006C006100620073000000040309040902EA
:100550005B00030100A0FA0904000001030101008F
:10056000092111010001224400070581030800014F
:100570000904010002030000000921110100012209
:100580002200070582032000010705030320000164
:1005900009040200010300000009211101000122E9
:1005A000B6000705840320000112010002000000CC
:1005B00008EBCE07000100010203010660FF09619C
:1005C000A1010962150026FF009520750881020926
:1005D00063150026FF00952075089102C0050109EA
:1005E00002A10185020901A10005091901290815C7
:1005F00000250195087501810205010930093115B1
:1006000081257F95027508810609381581257F951A
:100610000175088106050C0A38021581257F9501B0
:1006200075088106C0C005010980A1018503190173
:100630002AB700150126B700950175108100C00585
:100640000C0901A101850419012AA002150126A0A7
:1006500002950175108100C005010906A1018506FA
:10066000050719E029E715002501950875018102A4
:100670000507190029EF1500250195F07501810284
:100680000508190129059505750191029501750364
:100690009101C005010906A101050719E029E71527
:1006A00000250195087501810295017508810105F4
:1006B00007190029FF150026FF009506750881001F
:1006C00005081901290515002501950575019102F7
:1006D000950175039101C00011241FBECFEFDAE030
:1006E000DEBFCDBF12E0A0E0B1E0E4E5F8E602C075
:1006F00005900D92AC30B107D9F723E0ACE0B2E041
:1007000001C01D92A935B207E1F70E94EF120C94C7
:10071000AA3376CC862B81110BC0453048F4E42FE8
:10072000F0E0EE0FFF1FE455FF4F8591959108957E
:1007300081E090E00895811111C0653078F4E62FD2
:10074000F0E0EE0FFF1F81E04827E40FF11DEE0FF0
:10075000FF1FEA54FF4F85919591089581E090E045
:1007600008959C019A9581159F4118F5F32FF27019
:10077000EE27832F8170732F74706627532F587064
:10078000442734FF0CC08295807FEF2B09F08062F4
:10079000672B09F08064452B69F080680895EF2B82
:1007A00009F08260672B09F08460452B19F088609E
:1007B000089580E00895CF93DF93EB01D2DFFE012F
:1007C0000995DF91CF910895CF93DF93EC01805E7F
:1007D0009109089720F06FE578E0209711F46CE418
:1007E00076E0CE01E8DF8C2FC9D1DF91CF9108955B
:1007F000CF93DF93EC0106D2CE01805E910908977A
:1008000020F064E678E0209711F461E576E0CE010F
:10081000D2DFDF91CF91089581E0089581E00895BE
:10082000FBCF089581E0089581E0089581E0089567
:10083000FDCF089508950895FDCF08950895089572
:10084000A6E0B0E0E6E2F4E00C94533249835A8328
:100850009E833091130289819A81311117C03E81A4
:10086000311589F0211579F065D5182F682F898108
:100870009A8136D569817A81812F0E942F10269620
:10088000E3E00C946F3241D5182FF4CF53D5698132
:100890007A81F3CFFC01262F4081518162817381DF
:1008A00084819581CDCFCF93DF93D82FC92F61E07D
:1008B000F1DF6D2F7C2FB2DF811539F061E08D2FD4
:1008C0009C2FE8DF6D2F7C2FABDFDF91CF91089558
:1008D0000F931F93CF93DF93D82FC92F60E0DADFF8
:1008E0008C016D2F7C2FA7DF6D2F7C2FC801A4DF1B
:1008F000DF91CF911F910F91089591E001C0990F61
:100900008A95EAF7892F45C4CF93C82F81E00C2E32
:1009100001C0880F0A94EAF70E943B0E8C2FEDDF8E
:10092000CF91089581E0089581E00895FBCF089567
:10093000CF93C82FDFD38C2FF7DF8C2FF7DF2FEF6C
:1009400084E39CE0215080409040E1F700C000002B
:10095000CF91089581E0ECDF0C94C72A80E0E8DFB6
:100960000C94D82A0F931F93CF93DF93EC018B0144
:10097000FB01858181110E948619B801CE0154DFE7
:10098000811509F45BC0B801CE0152DF811509F46D
:1009900055C0B801CE010E948526811509F44EC0CC
:1009A000B801CE010E941A1B811509F447C0B80195
:1009B000CE010E94B525811509F440C0B801CE01D1
:1009C0000E94F1208115D1F1B801CE010E94C6200C
:1009D0008115A1F1B801CE010E940713811571F1B3
:1009E000B801CE010E94F525811541F1B801CE0173
:1009F0000E944C11811511F1F8018581811581F05A
:100A0000CA35FCE7DF0721F170F4C130ECE7DE07FF
:100A1000E9F0C330FCE7DF07B9F0C115DC4769F046
:100A2000C80100DF0CC0CB35ECE7DE07A1F0CC3508
:100A3000DC47B1F70E94FC0DF3CF8CDF80E0DF9143
:100A4000CF911F910F9108950E94300E87DFF6CF4E
:100A50000E94030EE5CF0E94050EE2CFCF93DF93F5
:100A6000D82FC92F61E016DF6D2F7C2F7BDFDF9140
:100A7000CF910895E3DE0E94092A17C018D0DFDE67
:100A80000C940D2A81E008950895CF93DF93D82F19
:100A9000F9DFC82F811511F08D2FF6DF8C2FDF9134
:100AA000CF9108950895F1CF089580E0FCCF0E9482
:100AB000EC27F9CFCF930E94EC27C82F80910E022C
:100AC0008C1771F0C0930E020E94972A60930F0258
:100AD0007093100280931102909312028C2FE3DF27
:100AE000CF910895ADE0B0E0E8E7F5E00C94523224
:100AF000488759876A877B878C879D8791116CD738
:100B00001F8226E0FE013896CE010196DC0101909D
:100B10000D922A95E1F720912C038C0122FF09C048
:100B20001DD7811519F082E00E94D50DFDD68111E7
:100B3000A3D78D8181110CC029813A814B815C81C1
:100B40006D817E818F8174D62D96E4E00C946E3297
:100B5000C801A9DE8111F0CFF7CFFC01848181307B
:100B600019F4808191810EC40895611521F00E94CD
:100B700053220C940C230E949422FBCFCF93C82FB6
:100B8000811589F08CEF8C0F813A78F48C2F0E94BC
:100B9000AC28811521F08C2F0E945129D7D78C2F9A
:100BA0000E943A29D3D7CF91089580E28C0F8830E4
:100BB00040F4C77081E001C0880FCA95EAF7EDD60E
:100BC000F1CF8BE58C0F833038F42C2F2452330B6C
:100BD000C9010E942E28E7CFE8E5EC0FEB3150F475
:100BE000F0E0EE0FFF1FEA5CFE4F808191810E94D2
:100BF0005628D9CF83E38C0F8331A8F661E08C2F80
:100C0000B4DFD1CF811551F19CEF980F913A18F4D0
:100C10000E9451299BC790E2980F983048F4877042
:100C200091E001C0990F8A95EAF7892FBCD6F2CFDF
:100C30009BE5980F933020F480E090E00C942E28F0
:100C400098E5980F9B3120F480E090E00C945628B2
:100C500093E3980F933110F460E087CF08951F93CA
:100C6000CF93DF93182FEB0189DF209731F4812F89
:100C7000C9DFDF91CF911F9108958FE99FE0019720
:100C8000F1F700C000002197F0CF60E570E08933F4
:100C900011F060E070E0E3CF811511F07ED656C709
:100CA0000895811511F07FD651C70895A0E0B0E0F6
:100CB000ECE5F6E00C944E326C01D62FC72FFC0108
:100CC0000581F6801F2D12951F705CD6E82E8115C8
:100CD000E9F0E02E0115D1F08C2F807F803461F097
:100CE00080E28D0F8830E0F08C2F807E803221F4FE
:100CF000D230B0F01115A1F080912C0382FF10C00A
:100D000082E053D73FD691E0E82EE926EC2FE2951A
:100D1000EF70C03C78F5F0E0E455FC4C0C941232D6
:100D2000E12CF4CF1C2F1F70C03110F01295107FF2
:100D3000011581F0111549F080E28D0F883010F017
:100D4000D11105C0812F29D601D78D2F42C0812F07
:100D500035D6FACF8D2F56DF111561F080E28D0F59
:100D6000883010F0D11103C0812F1DD602C0812F11
:100D70002BD6ECD6E11409F4C5C0ECD580FDC2C079
:100D8000F6011582E1D527D2C6017BD1DDD52DD262
:100D9000B9C0FC2FFF70FF2EC07FC03219F0F29453
:100DA00080EFF822D11549F0D13009F442C0011585
:100DB00009F44BC01115C9F0C8CF80912C0382FDF6
:100DC00010C0011541F0F11419F08F2DE6D5BED6F3
:100DD00080E0D4DECFCF80E015DFF11459F28F2D03
:100DE000C4CF0115A1F0111103C08F2D55DFC2CF63
:100DF000113019F48F2D11D6BDCF153009F0BACFAF
:100E00008F2D4ADF8F2D1FD68F2DECD5B3CF11112B
:100E100007C08F2D46DF8F2D16D68F2DEFD5AACF89
:100E2000113009F0A7CFB6D58F21811509F4A2CFD3
:100E3000F0CF011521F0163008F09CCFD6CF153039
:100E400008F098CF8F2D2DDF95CF1115D9F3D93319
:100E500049F42FEF87EE93E0215080409040E1F776
:100E600000C000008D2FCEDE85CF8C2F8695869515
:100E70008370811569F0813009F07CCF8D2F9C2F14
:100E80009370011102C080E090E00E94562872CF5A
:100E90008D2F9C2F9370011102C080E090E00E9482
:100EA0002E2868CF602F8D2F60DE64CF8C2F83704B
:100EB000811133C0011123C04D2F429546954770D3
:100EC000440F440F8D2F8F70042E01C0880F0A9499
:100ED000EAF72D2F2071D4FF07C02FE030E001C0CA
:100EE000220F4A95EAF72095C695C695C370822BC6
:100EF000C23079F0C33079F0C13049F050D10E944E
:100F0000EC27D1DDCDB7DEB7E8E00C946A3243D1EF
:100F1000F6CF49D1F4CF3DD1F2CF011531F1C0FF69
:100F2000EECF4D2F429546954770440F440F8D2FBD
:100F30008F70042E01C0880F0A94EAF72D2F2071BC
:100F4000D4FF07C02FE030E001C0220F4A95EAF736
:100F50002095C695C695C370822BC23059F0C33018
:100F600059F0C13029F05DD1CACF823040F2D9CFDB
:100F700054D1C5CF5AD1C3CF20D1C1CFCF70011525
:100F800029F08C2F28D18D2F87DEB9CF8D2F89DEC8
:100F90008C2F2BD1B4CFD23F31F168F4D03FC1F0C8
:100FA000D13F89F0011509F448C0111509F442C078
:100FB0008D2FE4DDA4CFD33FE1F0D43F99F78091AA
:100FC0002C0382FD1EC08C2F8F71011511F30FC0F1
:100FD000011539F0153008F092CF8C2F8F7113D195
:100FE0008ECF1630F8CF8C2F8F710111D2CFF3D066
:100FF00086CF011521F08C2F8F71E6D080CFE2D003
:101000007ECF011579F0A6D4843021F4C6D58C2F7B
:101010008F71BFCF63E0153008F071CF8C2F8F71C7
:10102000A2D56DCF153018F0B8D564E0F7CF81E0C8
:10103000BCD565CF8C2F8F71DACF111541F3D93321
:1010400049F4EFEFF7EE23E0E150F0402040E1F704
:1010500000C000008D2FD6DD52CF0F931F93CF938A
:10106000DF93EC01688179818D8197D18C01E1D08A
:101070008FD0B801CE011ADEDF91CF911F910F9171
:101080000895CF93DF93EC018C81811581F0CE011F
:10109000E5DC81110FC076D4811549F08D81811571
:1010A00031F080912C0382FF02C082E07ED5DF9177
:1010B000CF910895CE01D1DFCE010ADCF8CF8115A2
:1010C00011F07CD443C50895811511F07DD43EC53F
:1010D000089580E090E00E942E2880E090E00E9439
:1010E00056287AD433D50E9426230C940C230E94D0
:1010F0006829EFCF60D4FBCF282F92959F70963050
:1011000099F060F4925F9F70923030F4203FB1F01C
:1011100038F481E0283E38F080E008959A5FF3CFFC
:1011200081E0243FC9F7089591E0813F09F090E004
:1011300081E0283E08F080E0892B089581E0089541
:10114000FC018481811521F0808191811BD1D4CF54
:1011500080E00895A6E0B0E0E0EBF8E00C945432B3
:101160002696E2E00C947032A7E0B0E0EAEBF8E0FB
:101170000C9454322796E2E00C9470320895FECF1E
:101180000895FDCF0895FADFFCDF80931B020895D8
:101190000895F9CF089590911B02892BF4CF909177
:1011A0001B028923F0CF90911B028927ECCFE6CF59
:1011B0000895FDCF0895E2CF0895FDDFFADF809313
:1011C0001A02089580E0F9CF91E001C0990F8A9545
:1011D000EAF7892FF2CF21E030E001C0220F8A9593
:1011E000EAF780911A02822BE8CF21E030E0A901D2
:1011F00002C0440F551F8A95E2F7CA01809590916D
:101200001A028923DACF21E030E001C0220F8A954B
:10121000EAF780911A028227D0CF90911A02892B87
:10122000CCCF90911A028923C8CF90911A028927B6
:10123000C4CF08959B01677091E001C0990F6A9532
:10124000EAF763E0369527956A95E1F7B901660FED
:10125000771F260F371FFA01E20FF31F40E050E01F
:10126000682F70E08191DF019B01042E02C036954A
:1012700027950A94E2F7217021952827292328270A
:101280002E934F5F5F4F4330510561F708959C01E6
:10129000A82FA77083E0369527958A95E1F7C901B5
:1012A000880F991F820F931FFB01E80FF91F40E081
:1012B00050E080E0219130E00A2E02C0369527955B
:1012C0000A94E2F721703327042E01C0220F0A94FA
:1012D000EAF7822B4F5F5F4F4330510559F708956E
:1012E000282F862F903F41F0911107C0622F70E0A8
:1012F00047E152E0253040F008959C5F9230E0F7DE
:10130000622F70E044E152E095CF282F892F903F63
:1013100079F0911105C067E172E0253030F0089551
:101320008C5F823028F464E172E0822F90E0AFCFCE
:1013300080E00895A0E0B0E0E0EAF9E00C944F32DC
:101340007C0100911A0280911B02082BC3E0D0E0BF
:1013500010E0C8010C2E02C0959587950A94E2F71B
:1013600080FD09C02197A8F7D12C8D2DCDB7DEB710
:10137000E7E00C946B32DC2EB7018C2F96D60197E8
:1013800089F3F3CFCF93DF93D82FC92FD3DF6D2FFE
:101390007C2F8BD6DF91CF9108951F93CF93DF934E
:1013A000162FD72F90911302911539F0862F972F72
:1013B000E9DFDF91CF911F910895811569F0862FA4
:1013C000972FB8DFC82F682F812F9D2F89DF612FBE
:1013D0007D2F8C2F6AD6EDCF862F972F96DFC82FC3
:1013E000F6CFE1E0F0E0DF0102C0AA0FBB1F6A9573
:1013F000E2F7BD01DF0102C0AA0FBB1F4A95E2F769
:101400006A2B01C0EE0F2A95EAF7962F98239613C0
:1014100002C08E2B0895E0958E230895242F462F29
:10142000682F80911A02DDDFC8CE0F931F93CF93F0
:10143000E0911C02C7E080911D028E1304C0CF9181
:101440001F910F9108950E2F10E0CE9FF0011124EF
:10145000E25EFD4F2081318142815381648175813B
:10146000868182DEF8013196E770E5CF2091560241
:1014700030915702409158025091590260915A029E
:1014800070915B0280915C026FCE80915C02803132
:1014900078F480915B02811559F0E0911C02209153
:1014A0001D02309157024091560257E02E1301C0A1
:1014B00008956E2F70E05E9FF0011124DF01A25E9F
:1014C000BD4F14968C911497811549F111968C910A
:1014D0001197831324C08C91841321C015968C918D
:1014E000159781111CC012968D919C91A091580264
:1014F000B09159028A1B9B0B883C910580F4809126
:101500005C028F70806180935C02EC5DFD4F808196
:101510008F708061808386E592E0B3DD86CFFB012A
:101520003196E770C3CFE0911C0290911D0227E035
:10153000E91302C080E00895AE2FB0E02E9FF001C5
:101540001124E25EFD4F3181361306C0308138131D
:1015500003C03581341304C0FD013196E770E8CF34
:1015600081E008958F929F92AF92BF92DF92EF92A7
:10157000FF920F931F93CF93DF93CDB7DEB72D97D5
:101580000FB6F894DEBF0FBECDBF8C0186E0F80128
:10159000DE01189601900D928A95E1F7F801F58029
:1015A000848196E5892E92E0992E90915A029111AC
:1015B00017C0811509F4EFC0F11409F42EC1C80158
:1015C000BFDD811509F429C187E0F801D40101903C
:1015D0000D928A95E1F7C401C0DA57DF47DFDBC01F
:1015E000E080A280B380D0905B02209158023091BD
:1015F0005902A501421B530BD11409F4CFC0483C3A
:10160000510508F09EC0811509F4C5C0909157029C
:10161000918080915C02803108F065C0991226C0EB
:10162000909156029E1122C0F11057C08F708061B8
:1016300080935C021BDF86E592E023DD80915C02F3
:10164000F8018683F12C8F2D2D960FB6F894DEBF0E
:101650000FBECDBFDF91CF911F910F91FF90EF9003
:10166000DF90BF90AF909F908F900895F11035C09C
:1016700040E0692D8E2D57DF40E0692D8E2D53DF20
:10168000F82E8111DFCF888599857CDE292F229560
:101690002F70903450F49F70223078F0911591F0B3
:1016A000F8019681903170F4CECF2A5F2F702230EE
:1016B00070F0C801E6DCFD2CC6CF911519F081153C
:1016C00009F4C1CF805E883008F4BDCFF2CF803FEF
:1016D00008F4B9CF815F8330F7CF80915C028160DD
:1016E00080935C02AFCF991207C0909156029E1171
:1016F00003C0F11409F473C0C80122DD811509F497
:101700008CC0F11409F489C080915C02803280F0B1
:1017100020915602309157023A832983BC82AB82D2
:1017200090915A029D831E828F83CE010196A9DC7F
:1017300087E0F801A6E5B2E001900D928A95E1F705
:101740004CCF90915C02903188F4488559856A8528
:101750007B858C859D85FEDC86E592E092DC87E0CA
:10176000F40111928A95E9F781DE6CCF811599F029
:101770002091570281812813BFCF809156028E118C
:10178000BBCFF110B9CF9683C8017BDC87E0F401B1
:1017900011928A95E9F7FF24F39455CF483C5105FF
:1017A00008F03EC08115B9F3F114B9F190915702D8
:1017B0008181981329C0809156028E1125C0809195
:1017C0005C0280FD18C08031B0F08683807F803F4E
:1017D00039F08681982F907F905F8F70892B868358
:1017E000C8014FDC87E0F801A6E5B2E001900D9258
:1017F0008A95E1F7F3CE87E0F801A6E5B2E0019023
:101800000D928A95E1F7C7CFC8019ADC811190CF7C
:1018100080915C02816080935C02C80132DCBBCFA6
:10182000488559856A857B858C859D8593DC97CF16
:10183000AEE0B0E0EEE1FCE00C945332288739874B
:101840004A875B876C877D878E87CE0108968ADE04
:101850006C858115A1F0611539F0288539854A8597
:101860005B857D858E8580DC17E080911C029091E0
:101870001D02891338C02E96E3E00C946F3287E086
:10188000FE013896DE01119601900D928A95E1F7DE
:10189000611551F3A0911D028A2F90E00196877087
:1018A000992720911C022817190681F097E09A9F2A
:1018B000D0011124A25EBD4FFE01319601900D9220
:1018C0009A95E1F780931D02B0DDCECF13DC109224
:1018D0001D0210921C0287E0E6E5F2E0DF011D9296
:1018E0008A95E9F7C1CF189FC0011124825E9D4FF0
:1018F00039DE811509F4BFCFE0911C021E9FF00173
:101900001124E25EFD4F2081318142815381648147
:101910007581868129DC80911C0290E00196877098
:10192000992780931C02A1CF0E948B2A20918802C4
:1019300030918902AC01421B530B9A0181E0283897
:10194000334108F480E0089580918702869586955A
:101950008695089580918702877008950E948B2A4A
:101960002091850230918602821B930B8838934127
:1019700038F080918702002482FF0394802D08951F
:1019800080E0089590918702977081E0911101C0E5
:1019900080E008958091B50208959091B502982B4A
:1019A0009093B5020895982F90958091B502892360
:1019B0008093B50208951092B50208959091B402F3
:1019C000982B9093B4020895982F90958091B4022B
:1019D00089238093B40208951092B4020895089563
:1019E000FECF0895982F80918A02282F2923291746
:1019F00021F0892B80938A02F3CF089590918A0277
:101A0000292F2823211529F08095892380938A0284
:101A1000E7CF08950895FECF0895CF93C82F809102
:101A20008B028C238C1769F00E948B2A9093890279
:101A30008093880280918B028C2B80938B028C2F59
:101A4000EADFCF91089590918B02292F2823211549
:101A500079F08095892380938B02811551F00E9443
:101A60008B2A809388029093890280918B02D3CF36
:101A7000089580E090E0F5CF80918B02811541F0D0
:101A800010928B02109289021092880280E0C3CFDC
:101A90000895CF93C091B5028091B402C82B809174
:101AA0008B02811551F040DF8111E6DF80918B02BE
:101AB000C82B0E948B288111DFDF8C2FCF910895D6
:101AC000CF93DF93C0910601D0910701E2DF8883B5
:101AD000C0910601D091070148E050E06DE772E047
:101AE000CE010E941C33892B59F088E0FE01ADE73E
:101AF000B2E001900D928A95E1F7CE010E94FB279A
:101B0000DF91CF910895CF93DF93C0910401D091DD
:101B10000501BFDF8983C0910401D091050140E236
:101B200050E06DE572E0CE010E941C33892B59F024
:101B300080E2FE01ADE5B2E001900D928A95E1F7F9
:101B4000CE010E940828DF91CF9108950E94E527D9
:101B5000811529F080912B0387FF01C0D4CFB0CF2E
:101B60000895FECF0895962F20912C0322FF14C0D4
:101B7000682F660F660F660F692B609387022BDB59
:101B80000E948B2A9093860280938502809187021F
:101B9000869586958695E5CF1ECB1092870210928A
:101BA00086021092850280E0DCCF909187028095BA
:101BB000892380938702282F277021110BC0891752
:101BC00049F090912C0392FF05C0869586958695E5
:101BD0000CDBE3CF089590912C0392FB222720F990
:101BE000281749F080FB92F990932C038BE293E045
:101BF00046D082E0DACF089580912C03002482FF42
:101C00000394802DE8CF81E0E6CF80E0E4CF60E070
:101C100070E0CB01FFC360E070E0CB01F5D3F7CFFC
:101C2000A3E0B0E0E6E1FEE00C94543247D352D397
:101C30001B82CE01039665D381E080931B026BD398
:101C4000198284E18A83CE01019676D3EAD50E9477
:101C50007126E1DF2396E2E00C947032E1CF089523
:101C60003FC308952CD381110C94292608953EC3B7
:101C700008954DC308954FC3089552C308955CC39A
:101C8000089561C30895A0C30895CAC30895A6E046
:101C9000B0E0EDE4FEE00C9452320E948B2A8C01FD
:101CA0008091B6029091B7028017910779F019825E
:101CB0001A820E948B2ABC0149815A8180E090E0FF
:101CC0000E9472051093B7020093B6022696E4E0D4
:101CD0000C946E320E94972A6093C1027093C202E4
:101CE0008093C3029093C4026093BD027093BE02BE
:101CF0008093BF029093C00208950E94972A609338
:101D0000C1027093C2028093C3029093C402609395
:101D1000B9027093BA028093BB029093BC020895FB
:101D200008950895FDCF08950895FEDFFBCF08952F
:101D3000FECF08950895FEDFFBCF8AE491E162D4DF
:101D40000E948C19EEDFF1CF81E0089581E00895C3
:101D5000FBCF0895089508950895FCDFFCDFFCCFC4
:101D600081DF811101C07ADF85EC92E080DF8BE2B8
:101D700093E083DF0E94061D7CDF0BDA80911A025C
:101D800018CA0E94822A0E947D260E941F1BBBD374
:101D9000E7DF0E9452050E94B118CDCFA6E0B0E067
:101DA000E4EDFEE00C944F32D1DF81110FC06FDF04
:101DB0000E9487190E948A1B81119FDF0E9447237E
:101DC0000E945A052696E7E00C946B32A4D310913A
:101DD000B80280E044D3181751F38091C50281FD09
:101DE00044D3B6DFD82E80E03AD3182F9091B802B2
:101DF000891731F1E82EE92600E0FF24F3948E2DB7
:101E00008F218115B9F0D114A9F009831A820E949B
:101E10008B2A9C838B8381E08D8391E0812F8F219E
:101E2000811101C090E049815A816B817C818D8153
:101E30000E9472050F5FFF0C053009F71093B8027E
:101E400049DFB6CF1F93CF93DF9331D1EC018115DA
:101E500022E5920708F05AC0811540E5940708F082
:101E6000D7C0803E910528F58D3C910508F0A9C0AA
:101E7000883A910578F4853A910508F09FC0813041
:101E8000910509F43EC00497813A9105D0F1C0E074
:101E9000D0E037C0885A91094B97C8F7C85AD0E0AC
:101EA000CC0FDD1FC459DE4F0990D881C02DD464FA
:101EB00028C0811550E49507E8F4C11580E2D807E1
:101EC00008F0BCC0C83ED105E0F0CE019A9581155E
:101ED0009F41E8F68D2F8FD1182FCE019927E7D09B
:101EE000212F30E0322F2227E901CC27DF71C82BC8
:101EF000D92B07C09927DBD0CC27DF70C82BD92B73
:101F0000D06ACE01DF91CF911F910895803842E5CC
:101F10009407C8F5803652E5950708F05BC0C034D9
:101F200082E5D807D0F4C03292E5D90708F04BC05B
:101F30008C2F8695869520E2829FC0011124C37064
:101F400021E030E0A90102C0440F551FCA95E2F715
:101F5000EA01C82BD92BDD68D4CF8C2F86958695C6
:101F6000877050E2859FC0011124C37021E030E0EA
:101F7000A90102C0440F551FCA95E2F7EA01C82B18
:101F8000D92BDC68BECF803C52E5950758F48F71A1
:101F9000C03AD245A0F590E0982F8827EC01C46F95
:101FA000D06AAFCF805C9245809708F070CFDC2F6D
:101FB000CC27CC27DF71C06FD06AA3CFA497D064A1
:101FC000A0CFD0659ECFCF71D0E0DC2FCC27C16FE2
:101FD000D06A97CF86958695877020E2829FC00150
:101FE0001124C37021E030E0A90102C0440F551F45
:101FF000CA95E2F7EA01C82BD92BDA6882CFFBD069
:10200000C82FD0E0DC2FCC27CC27DF71D06279CF6E
:102010008F71F1D053E0CC0FDD1F5A95E1F7CC273B
:10202000DF70282F30E084FF05C050E1859F9001CC
:1020300011243327C22BD32BD06963CF8D2F8F71FF
:10204000DAD0182FCE01992732D0212F30E0322F4D
:10205000222722273F71282B392BE901D7CF209146
:10206000F1023091F202232BB1F4703F39F4603F5A
:1020700091F480913703909138030895711106C04F
:10208000653048F4462F60E00C94811D7D3F31F4AB
:1020900041E0653040F080E090E008957C3FD9F762
:1020A0006530C8F740E00C948B1DD9DFCBCE803E65
:1020B0009105D9F1C8F48133910509F482C048F43F
:1020C0008932910509F472C08A32910509F480C001
:1020D000089589339105E9F082389105D1F085336F
:1020E000910509F45EC00895843E9105D9F148F444
:1020F000823E910539F1833E910549F181EE90E0F0
:102100000895863E9105C9F1873E910509F43EC0C8
:10211000089520912B032370211164C020912C037A
:1021200023FF14C089E290E0089520912B0320FD45
:1021300045C030912C0330FF09C024FD24C083EE3C
:1021400090E0089520912B0322FDF7CF0895209170
:102150002B0322FD44C030912C0330FD43C024FFEB
:10216000F5CF11C020912C0321FFF0CF80912B03DC
:1021700084FD09C087EE90E0089520912B0323FF92
:10218000E5CF24FFF7CF80E090E0089520912B0366
:1021900023FD2BC030912C0331FFE1CF84EE90E082
:1021A000089520912B0325FFD1CFBCCF20912B0385
:1021B00025FD1EC020912C0323FFC8CF89E390E0AA
:1021C000089520912B0326FFC1CF8AE290E0089565
:1021D00020912B0326FFBACF81E390E0089582EE91
:1021E00090E0089580EE90E0089586EE90E00895E6
:1021F00085E390E0089590912B0392FF10C041E099
:10220000282F2471243009F040E031E0282F287174
:10221000283009F030E0431711F02CE0822793FFBB
:1022200010C041E0282F2471243109F040E031E052
:10223000282F2871283109F030E0431711F02CE0E5
:10224000822730912C0330FF10C051E0282F2171DC
:10225000213009F050E041E0282F2871283009F0A2
:1022600040E0541711F029E0822731FF10C041E00F
:10227000282F2171213109F040E031E0282F287109
:10228000283109F030E0431711F029E0822794FD4E
:10229000877E089580E00895CF939C01FB01805EC6
:1022A0009245C1E0809738F4C581C11104C0822FE6
:1022B0008F710E9484048C2FCF910895089580E03F
:1022C00090E00E9446339C0181E0233E3E4F09F09E
:1022D00080E0089563EE7EEF80E090E00C9474332C
:1022E0006FEF7FEF80E090E00C947433CF93DF9337
:1022F000EC0182E090E00E9439338883DF91CF9136
:102300000895FC01608182E090E00C945A3383E0F0
:1023100090E00C943933682F83E090E00C945A33AA
:10232000CF93DF93EC0184E090E00E9446339983E1
:102330008883DF91CF910895FC016081718184E0F1
:1023400090E00C9474338F929F92AF92BF92CF9291
:10235000DF92EF92FF920F93CF93DF93EC0188E02F
:1023600090E00E9441334B015C0168839982AA820C
:10237000BB821C821D821E821F8283E290E00E942B
:102380003933282F30E040E050E060E070E080E03A
:1023900090E000E20E947B32282939294A295B29F2
:1023A000288339834A835B836C837D838E839F83F9
:1023B000DF91CF910F91FF90EF90DF90CF90BF9082
:1023C000AF909F908F9008950F93CF93DF93EC0180
:1023D000488159816A817B8188E090E00E946C335A
:1023E000288139814A815B816C817D818E819F81C9
:1023F00000E20E949632622F83E290E00E945A33FC
:10240000DF91CF910F910895AB01BC018FE090E077
:102410000C946C33AB01BC0183E190E00C946C3301
:10242000682F8EE090E00C945A330895FECF089503
:102430000895FECF0895E82FF0E0E25DFC4F808123
:1024400090E021E030E002C0220F331F6A95E2F7EE
:102450002823392381E0232B09F480E00895E82F15
:10246000F0E0E25DFC4F808108950895A2EAB1E0BA
:1024700021E030E08D918F3FA1F0E82FE295EF70E1
:10248000F0E041A18F70B90102C0660F771F8A95F5
:10249000E2F7CB01962F9095942391A392A1892BDB
:1024A00082A371E0A73AB70729F70895CF93DF9386
:1024B0009C01C62FD0E085E0689FF0011124EE5505
:1024C000FE4F65E071E050E041914F3F79F0A42F5D
:1024D000A295AF70A05EB0E08C9190E04F7002C00A
:1024E000959587954A95E2F780FF0BC080E0582BC1
:1024F000770F6A9549F7C20FD31F5883DF91CF91A9
:102500000895872FF4CFB2DF10922E0310922D037F
:1025100081E023D08BCFA1E0B0E0E1E9F2E10C94BF
:102520005332198260E0CE010196C0DF90912D03F5
:10253000898121E098130EC020E041E06EE273E053
:102540008DE293E00BD0182F74DF812F2196E3E00A
:102550000C946F3280932D03F0CF0895A0E0B0E08B
:10256000E4EBF2E10C944E32D82EE92EF62ED72F62
:10257000042FC22F211579F081E08093C8020E94B8
:102580008B2A9093C7028093C60280E0CDB7DEB756
:10259000E8E00C946A32C090C802C114B1F3809193
:1025A000C6029091C7020E941C2A059770F310E0A2
:1025B000A8016D2D7E2D8F2D9D2F0E941C33892B00
:1025C00041F0A8016D2D7E2D8F2D9D2F0E94293366
:1025D000CC2D1092C8028C2FD9CFE0CB08950E9449
:1025E000252A0E94482CA9DB0E94602CCADB0E948D
:1025F000692C0E946C2CF1DF0E94822C0E94342BEB
:10260000ACDBF7CF90930D0280930C020895CF932B
:10261000DF93EC01FB018581811104C081E0DF9132
:10262000CF910895B7D98272FE01E052F847EB309E
:10263000F105A0F7E854FC4C0C9412328AD580E0E6
:10264000EECF811521F079D5FACF8115E1F36AD566
:10265000F6CF811521F03ED2F2CF8115E1F330D2D1
:10266000EECF811521F050D2EACF8115E1F33FD2B0
:10267000E6CF811521F062D2E2CF8115E1F351D28C
:10268000DECF811521F0FDD0DACF8115E1F3EAD05C
:10269000D6CFCF92DF92EF92FF921F93CF93DF932B
:1026A000172FE82F711111C0411521F0F0E0EC5106
:1026B000FE4FE4916E2F7E2F8E2FDF91CF911F91D1
:1026C000FF90EF90DF90CF900895C62ED12CE72E8B
:1026D000F12C411521F0F0E0EC51FE4FE49186E041
:1026E000689F90011124CFEFD0E0C901BE010E9484
:1026F000C931AB01C601880F991FF5E5F49FB00100
:10270000F59F700D1124861B970B682F660F680FBD
:102710006E01CE18DF08EC9DD001ED9DB00D1124A7
:102720009B2F169F60011124CD2CDD247E01EC1817
:10273000FD086701EC9D7001ED9DF00C11246E0108
:10274000C61AD108B601169F6001179FD00C11243C
:10275000CD2CDD24CC19DD09EC9F6001ED9FD00C60
:1027600011247D2D43305105C1F02C3F334050F4EE
:1027700041305105B1F04230510561F47E2FEB2F0D
:102780009D2D08C04430510579F04630510511F0B7
:102790007B2F9F2D6E2FE92F8FCF7F2D9E2FEB2F1D
:1027A000F9CF7E2FEF2DF6CF9E2FED2D7B2FF2CF81
:1027B00041E06FCF0895FCCF089590910B01291B44
:1027C000922FE091D401F091D501242F462F682F4C
:1027D000892F90E009950895CF93DF93982F762F56
:1027E000842FD22FC32F692FE6DF962F672F482F14
:1027F0002D2F3C2F892FE1DFDF91CF91089580911C
:102800002F03843028F48370846080932F0308950D
:102810008C3AE8F38370886AF8CFF1DF8FE293E0B7
:1028200032CAEFE2F3E085E0808311828FEF82838A
:1028300083831482CF0127CA80912F0380FF03C0B6
:1028400086958695089580E008959091330393309E
:1028500018F49F5F90933303811519F08FE293E092
:1028600012CA089581E0F1CF90913303911519F0C8
:10287000915090933303811519F08FE293E003CACE
:10288000089581E0F1CF809133030895809333035D
:1028900008958091300308958091310308958091C7
:1028A000320308950F931F93CF9380912F0380FFDE
:1028B00009C0E091D801F091D9010995CF911F91FC
:1028C0000F910895C0910D010091D4011091D5018F
:1028D00080910E01C81768F780910B019C2F981BFF
:1028E000892F20E040E060E090E0F8010995CF5F9B
:1028F000EFCFEF92FF920F931F93CF93DF93D82FD9
:10290000162F042F80912F0380FF0BC0C0910D0163
:10291000E090D401F090D50180910E01C81730F0FD
:10292000C1DFCDB7DEB7E6E00C946C3280910B01CD
:102930009C2F981B892F202F412F6D2F90E0F7019E
:102940000995CF5FE9CF982F762F842F20912F0301
:1029500020FF07C0692F2FDF962F672F482F892F61
:10296000C8CF0895CF93DF93EC01EC81F0E0E15202
:10297000FF4F4491EFE2F3E062818181E4DF8C81DB
:102980008F5F8C83DF91CF910895CF93DF93EC011C
:10299000EFE2F3E0438162818C81D5DF8C818F5F30
:1029A0008C83DF91CF910895CF93DF93EC01209139
:1029B00032039C81892F817090FD822F692F627074
:1029C00091FD622F492F447092FD422F92DF8C813E
:1029D00090E00196877099278C83DF91CF910895BD
:1029E000A0E0B0E0E6EFF4E10C944F32D82F062FD0
:1029F000142FE22E90912F0390FF21C0E92FE6952E
:102A0000E695AE2FB0E0A955BE4F8C918093EB02B6
:102A10009C7F9430C9F46D2F702F842FCCDE962FBD
:102A2000672F482F892F65DFD09330030093310340
:102A300010933203E11419F08FE293E024D9CDB75B
:102A4000DEB7E7E00C946B32823019F41091320358
:102A5000EBCF863019F4D0913003E6CF8930D9F32B
:102A6000893111F7E9518E2F8170D82EE695F0E06B
:102A7000E152FE4FC491F12C60910F01F61610F057
:102A800011DFD2CFFC9EC001112470E00E94C93139
:102A90008D2FD1100BC0860F20910D012F0D3327E4
:102AA000331F412F602F98DEF394E6CF861BF4CFBF
:102AB000282FEFE2F3E0818143816281885F90CF2C
:102AC00081E0F6CF282FEFE2F3E08181438162813C
:102AD000885086CF81E0F6CF282FEFE2F3E06281C5
:102AE00031E1630F08F46FEF4381818179CF81E099
:102AF000F3CF282FEFE2F3E0628131E1631B08F4AA
:102B000060E0438181816CCF81E0F3CF282FEFE239
:102B1000F3E0438131E1430F08F44FEF628181819B
:102B20005FCF81E0F3CF282FEFE2F3E0438131E183
:102B3000431B08F440E06281818152CF81E0F3CFF2
:102B400020E04ECFEF92FF921F93CF93DF93EC01E3
:102B500010E0EE24EA94F12C60910F01161768F052
:102B6000A1DE8C819A8190FF1DC08F5F8C83DF91E5
:102B7000CF911F91FF90EF90089520910D01210FAB
:102B80003327331F70E0C7010E94DD31962F8C81FF
:102B90004091320360913103199F800D11241CDE96
:102BA0001F5FDACF8150E2CFA0E0B0E0EAEDF5E1BF
:102BB0000C944D32FC018281D1E080FDDFEFC0E05A
:102BC000C090D401D090D50180910F01C81790F02A
:102BD00069DE8091CA02D13009F04BC0811102C078
:102BE00080910F0181508093CA02CDB7DEB7E9E032
:102BF0000C94693280910D0190910B01891B8C0F0F
:102C000020E040E060E090E0F601099504E010E08B
:102C1000B12CEC2EF12C8091CA028B0D86301CF168
:102C200065E00E94BC31892F082E001C00088E151B
:102C30000F0499F480910D019701280F311D4091E7
:102C400032030403A00111245595479555954795E6
:102C50006091310380913003BFDDBD0E0150104003
:102C6000D1F6CF5FB1CF87FFDFCF90910F01890FF2
:102C7000DBCF90E0019660910F0170E00E94DD31A2
:102C8000B2CF0F931F93CF93DF93C0910D010091AB
:102C9000D4011091D50180910E01C81750F110E0B8
:102CA000C091D401D091D50160910F01161770F138
:102CB000F9DD809109019091C902980F9093C902A2
:102CC00020910A01280F20930A01121654F4209132
:102CD0000F012150330B092E001C00089217030628
:102CE0001CF0819580930901DF91CF911F910F9185
:102CF000089580910B019C2F981B892F20E040E0C4
:102D000060E090E0F8010995CF5FC5CFE12FF0E0DA
:102D100070E0CF010E94DD3120910D01820F909172
:102D2000C902092E001C0008E917F0059CF09091DB
:102D30000A01092E001C00089E170F065CF0282FC0
:102D400030E040913203609131038091300344DDE3
:102D50001F5FAACF90910B01891B20E040E060E04B
:102D600090E0FE010995F4CFA6E0B0E0EAEBF6E1D1
:102D70000C944E328D839E83AD81BE811496FC915E
:102D80002F2F30E0D9010E9425329B01AC010E9417
:102D90003A326B017C0180E290E09C012F1B3109EB
:102DA000F901A5E5B0E0A70196010E943A326983D6
:102DB0007A838B839C839F01DF010E941F329B01DA
:102DC0000E9434329B01AC012C0D3D1D4E1D5F1D38
:102DD00069817A818B819C810E94F031022F30E0E1
:102DE0000A3240F5A901440F551F420F531F559554
:102DF0004795142F1095F12C85E5E82EE01A809167
:102E00000F01F81628F14EDDAD81BE8114969C911C
:102E100081E0911519F0903219F48FEF8093080139
:102E200080910801890FED81FE8184832696E8E078
:102E30000C946A3285E590E0821B930BAC01440F41
:102E4000551F480F591F57FFD2CF4F5F5F4FCFCF4E
:102E50008E2DF1FC802F20910D012F0D3327331F74
:102E6000412F60913103B8DCF394C9CF0F931F93C6
:102E7000CF93DF93EC0100E010E090910F01091770
:102E8000110564F00FDD8C8190E001968170992727
:102E90008C83DF91CF911F910F9108954C81809188
:102EA0000D019801280F311D60913103809130038D
:102EB00096950917110544F4411541F040913203EC
:102EC0008BDC0F5F1F4FD9CF4115C1F340E0F8CF26
:102ED000A0E0B0E0EEE6F7E10C944632FC0162803F
:102EE000448081E08483EFEDF0E07490EEE5F1E062
:102EF000E491C0913203C695C158D0E0CC0FDD1FDC
:102F0000CD2FDD27812C25E0922EAA24AA94B12C66
:102F100055245A94E719EE2EF12C80910F01881652
:102F200030F0C0DCCDB7DEB7E0E10C946232C82CE3
:102F3000D12C83E0681658F4989CF0011124E553D5
:102F4000FD4F809130038083809131038183411054
:102F50001BC09C9CF0019D9CF00D1124E553FD4F7E
:102F60001382128280910D019601280F311D9C9CC5
:102F7000F0019D9CF00D1124E553FD4F42816181CC
:102F800080812ADC8394C9CF9C9C80019D9C100D7C
:102F9000112405531D4FF80183818115F1F08150F3
:102FA0008383589EC0011124648170E00E94C9315E
:102FB000FB01FF27E152FF4F8491E82FE7195E9E46
:102FC000C0011124B7010E94C93180913203689F6A
:102FD000B0011124F8017283C5CF0E94F832B50107
:102FE0000E94DD318C179D070CF0BCCFF3E06F160B
:102FF00098F00E94F832B5010E94DD31F80180831B
:103000000E94F832209131032695622F70E00E94D1
:10301000DD31280FF80121839C9CF0019D9CF00D6F
:103020001124E553FD4F128280913203893C58F000
:1030300088EC9C9CF0019D9CF00D1124E553FD4F04
:10304000848383838FCF8431A0F784E1F2CFEFE2D2
:10305000F3E080818E7F8083CF010E94430E109227
:10306000EC0220CCEFE2F3E080818E7F808310922F
:10307000EC0218CC60912F036695669570E04BE0EA
:1030800050E080E191E00E940F33892B19F481E038
:103090008093EC020E948B2A9093E5028093E402D5
:1030A000089590912F0390FF2CC0811559F18B3218
:1030B00058F58F73880F880F90912F039370892B89
:1030C00080932F03611521F08FE293E00E94430E5D
:1030D00060912F036695669570E04BE050E080E1CB
:1030E00091E00E940F33892B89F01092EC0281E06D
:1030F0008093E70240913203609131038091300365
:103100001FCD089581E0D6CF8AE2D4CFB3DFEFCFD1
:10311000682F80912F03869586958F5F8B3208F0FC
:1031200081E0BFCF81E0F4CF682F80912F03869597
:1031300086958A9509F48AE2B4CF81E0F5CF61E003
:10314000B0CFEFE2F3E08081816080838695869541
:10315000F6CF80912F0380FF01C079CFF2CF60E0DE
:10316000A0CF8091EA0281111FC08FE293E00E94FC
:10317000410E80912F03843028F453DB8FE293E0DB
:103180000E94410E3CDB1092EC02E091D201F091E2
:10319000D301099580912F0380FF03C08695869502
:1031A000DEDF81E08093EA020895EFE2F3E08081C0
:1031B0008160808386958695D2CF0F931F93CF939E
:1031C000DF938091EC02811509F441C08091EB02FC
:1031D000E0912F03E695E695E81BE093E602853142
:1031E00009F48BC008F044C0893009F47CC0A0F514
:1031F000823009F466C0863009F46CC0C0EDD7E0B7
:103200000AED13E18091E702811561F01092E70267
:103210000E948B2A9093E5028093E4021092E902C7
:103220001092E8020E948B2A2091E4023091E5027C
:10323000821B930B8F3F9F4750F42C0F3D1F309301
:10324000E5022093E40284EE92E0F8010995DF9113
:10325000CF911F910F9108958F3081F6E695F0E0A0
:10326000EE52FF4FE491CE2FD0E004ED15E1CACF2E
:10327000C4EFD1E006E317E1843221F288F4C8E21A
:10328000D0E004EB16E1883109F4BCCF833209F0B9
:10329000B5CFEDECF0E0C591D59104ED14E1B2CFDE
:1032A000853209F0ABCF8E2F63E00E94B031E92F59
:1032B000F0E0E653FF4FE491CE2FD0E008E617E1AF
:1032C000A1CFF0E0E552FF4FE491CE2FD0E002EB2A
:1032D00014E198CFF0E0E852FF4FE491CE2FD0E018
:1032E00005EC14E18FCFE695F0E0EB52FF4FE4914F
:1032F000CE2FD0E002EA15E185CFF0E0E153FF4F99
:10330000E491CE2FD0E001E416E17CCF089555CFB3
:1033100008950C947E2808950895A8E0B0E0E3E9AC
:10332000F9E10C9450328C01603239F5DC011196D0
:10333000EC911197EE3008F5F0E0ED53FC4C0C9455
:10334000123288E0EAEDF1E0DE01119601900D9273
:103350008A95E1F7F80131968FE1DF011D928A9598
:10336000E9F786E0F801808388E0FE013196D80114
:10337000149601900D928A95E1F72896E6E00C9458
:103380006C3280E68C9381E011968C9311971296A3
:103390001C92129713961C92F0CFFC0182819381AC
:1033A000092E000CAA0BBB0B25E0880F991FAA1F42
:1033B000BB1F2A95D1F7AC01BD01405E5F4F6F4F37
:1033C0007F4F481759076A077B07B8F28036F1E04C
:1033D0009F07A105B10588F6413621E05207610536
:1033E000710520F040E651E060E070E0481B590BA9
:1033F000BC016C517D4FC8010E940633BECF1296AE
:10340000FC9012971396EC9040E06E2D8F2D19D3FF
:10341000982789279827F8019183808341E06E2DB2
:103420008F2D0FD3982789279827D80113969C931F
:103430008E931297A2CFFC01258136812C3731055E
:1034400079F032272327322741E0D80114968C9156
:10345000811101C040E0F80163818281F4D28DCFF7
:103460008091F3029091F40220E03CE7892B61F710
:1034700020E030E0E9CF4FE150E06FEF70E00196DF
:103480000E9432338091F302D8018C938091F10233
:1034900011968C93119712961C92129713961C9268
:1034A000139714961C92149784E015968C9365CF0D
:1034B00081E090E09093F2028093F10282E390E049
:1034C0009093F0028093EF020E948B2A9093EE0279
:1034D0008093ED0252CF8091F1029091F202892BFC
:1034E00091F160E080E00E941B12E82E64E080E031
:1034F0000E941B12F82E8091ED029091EE020E9424
:103500001C2A8536910550F1E11441F1F11431F195
:103510000E948B2A9093EE028093ED028091EF023D
:103520009091F00201979093F0028093EF02892B23
:1035300051F41092F2021092F10281E090E0909327
:10354000F4028093F3028091F302F801808380916A
:10355000F10281838091EF0282830FCF82E390E0BA
:103560009093F0028093EF02EECF1092F40210924B
:10357000F30203CF40E250E06FEF70E00E9432337D
:10358000FCCE12968C918111F8CE80E2F801119256
:103590008A95E9F7F2CEA6E0B0E0E1EDFAE10C940D
:1035A00054329093380380933703811520E29207B9
:1035B00030F40E94E4032696E2E00C94703280EF2F
:1035C00089838A830E948B2A8160BC0149815A8148
:1035D00081E091E00E947205EECFA6E0B0E0E3EF5B
:1035E000FAE10C9454329093380380933703811599
:1035F00020E2920730F40E94F8032696E2E00C9451
:10360000703280EF89838A830E948B2A8160BC019B
:1036100049815A8181E090E00E947205EECFCF93FC
:10362000DF93D82FC92FB7DF8D2F9C2FD6DFDF91E7
:10363000CF91089581E008950C94A40E0895E6EFCB
:10364000F2E08AE0DF011D928A95E9F727C1FC01CB
:10365000828190E0019666E070E00E94C9319C0191
:10366000938181E09217130609F080E008950F938B
:103670001F93CF93DF93EC01162F042FE8DF811106
:1036800018C0EA818E2F90E0EC0FFD2FF11D00FB9A
:1036900017F91483019666E070E00E94C9318A83AD
:1036A00088818F5F888381E0DF91CF911F910F9197
:1036B000089580E0F9CFCF93DF93FC01EA01A38165
:1036C00082818A17D9F0AE0FBF2FB11D14968C914D
:1036D00087FB992790F98F77DB018C9398838381FF
:1036E00090E0019666E070E00E94C9318383818199
:1036F0008F5F818381E0DF91CF91089580E0FBCFE0
:10370000462F682F86EF92E0B2CFAB01BC0186EF67
:1037100092E0D1CFAEE0B0E0E0E9FBE10C944E32B4
:103720008091F502811551F01092F5028091F80216
:103730008093F9028091F6028093F702E9D07CDF52
:10374000E82E811569F1E12C0CEF8DEFF82E1FC0EA
:10375000CD84DE84D982C11441F1FA820E948B2A81
:1037600032E0E32EBC0149815A818E2D91E00E9406
:103770007205DF82C114F9F0F8860E948B2ABC0121
:103780004F8158858E2D90E00E947205E12EBE017A
:10379000635F7F4FCE010E96B8DF182F8111D8CF0F
:1037A0008E2D2E96E8E00C946A320A830E948B2AB2
:1037B00023E0E22ED7CF0887E0CF8FE891E0019792
:1037C000F1F700C00000089590E06115E9F08D5018
:1037D0009E4FFC0180818F3FB1F0E82FE295EF70A2
:1037E000F0E041A18F7021E030E0B90102C0660F26
:1037F000771F8A95E2F7CB01962F9095942391A39A
:1038000092A1892B82A3089588509E4FE2CF90E029
:103810006115A9F08D509E4FFC0120812F3F91F042
:10382000E22FE295EF70E05EF0E0808190E02F7093
:1038300002C0959587952A95E2F781700895885082
:103840009E4FEACF80E008950895CF93DF93C0E0C4
:1038500080910003C81750F0B0DFC0E080910003F2
:10386000C81760F0F1DFDF91CF91089560E08C2FF1
:10387000ABDF61E08C2FA8DFCF5FEACF60E08C2F59
:10388000C6DFD82F61E08C2FC2DFEC2FF0E0EA5FBB
:10389000FC4F880F8D2B8083CF5FE0CF85E0809336
:1038A0000003D3CF1F93CF93DF93182F440F642BC4
:1038B000C82FD0E0DE01AA5FBC4FEC918E2F837041
:1038C000681711F1EE0FEE0FE62BEC93EF70F0E0BE
:1038D000ED51FE4FCF5FDC4F90818881980F988328
:1038E00092301CF060E0812F0BDF88818F3F1CF449
:1038F00061E0812F05DF8881082E000C990B62E0C2
:1039000070E00E94DD318883DF91CF911F9108958F
:10391000CF93DF93C0E080910003C81718F0DF91C8
:10392000CF91089561E08C2F72DFD82F60E08C2F4B
:103930006EDF682F4D2F8C2FB5DFCF5FECCF259A30
:103940000895FC01EE0FFF1FE80FF91FE75CFC4F25
:103950006183408322830895FF920F931F93CF9337
:10396000DF93182F062FF42EC0E0D0E02F2D402F2C
:10397000612FCE01E6DF2196C530D105B9F7CDB76D
:10398000DEB7E5E00C946D3235B13F7D25B12062A4
:103990004FB7F89489E393E0FC010196508168E009
:1039A00025B9000000C057FF35B9550F000000C011
:1039B00000C000C035B900C06A9591F753E0883463
:1039C000950751F74FBF8FE594E00197F1F700C0DD
:1039D000000008950C94300E089580E00E942F128C
:1039E000817008950E948B122FEF86E791E021509D
:1039F00080409040E1F700C000000E948B12EDDF94
:103A0000811519F0E7DF0C94C72A0895EBCF0895CC
:103A1000A1E0B0E0EEE0FDE10C9452328E010F5FC8
:103A20001F4F21E030E040E050E0EFD28981219645
:103A3000E4E00C946E3284E0089571C1089599C158
:103A40000895B9C10895EFC108950F931F93CF93BF
:103A5000DF930091F3021091F40281E090E09093E3
:103A6000F4028093F30259D1C0E0D0E04D2F60E022
:103A70008C2F0E948A039C014D2F60E08C2F79D1FE
:103A8000DF5FD53099F7D0E041E06D2F8C2F0E9499
:103A90009B039C0141E06D2F8C2FC5D140E06D2F21
:103AA0008C2F0E949B039C0140E06D2F8C2FBBD17B
:103AB000DF5FD53049F7CF5FC430B9F61093F40219
:103AC0000093F302DF91CF911F910F9108950F930F
:103AD0001F938A019B0140E050E0BC0180E090E030
:103AE000D3D11F910F9108950F931F938A019B01CA
:103AF00040E050E0BC0180E090E0F2D11F910F91D6
:103B00000895843028F4611103C0453008F407C1DA
:103B100080E090E00895843018F4653008F44BC1DB
:103B200080E090E0089580E108956AD2CB01089585
:103B30000F931F938A019B0140E050E0BC0180E09D
:103B400090E063D21F910F9108950F931F938A0104
:103B50009B0140E050E0BC0180E090E09AD21F91D0
:103B60000F910895DBD0D8C2A4E0B0E0EAEBFDE10C
:103B70000C944532182F803108F0CBC041D26150EF
:103B800071098109910944DF8111C3C039D24B0108
:103B90005C01C12CD12C760111113FC034E0332ED1
:103BA0008E010F5F1F4FF801232D11922A95E9F71F
:103BB000460157014FEF841A940AA40AB40AC701B8
:103BC000B60126DF8983811509F4A3C0813009F08D
:103BD0009CC02601370152E0450E511C611C711C2E
:103BE000C501B40115DF8A83811509F492C09FEFE6
:103BF000980F933020F5C301B2010ADF8B83811542
:103C000011F0C8014CD74601570183E0880E911C82
:103C1000A11CB11C75016401C6CF8C149D04AE04B7
:103C2000BF0409F476C0C701B601F2DE2FEFC21A55
:103C3000D20AE20AF20A8111F0CF1150ADCF9BEF08
:103C4000980F933078F54601570193E0890E911C47
:103C5000A11CB11CC301B201DBDE8B838115D1F243
:103C6000E4E0CE0ED11CE11CF11CC501B401D0DE94
:103C70008C83811581F08B819C818130FFEF9F07C0
:103C800010F0982F88272A81263041F0273041F004
:103C9000253009F4C4DC46015701BCCF7CDCFBCFE6
:103CA0009CDCF9CF53014201843009F0B3CFC3014A
:103CB000B201AEDE782E4601570124E0820E911C3F
:103CC000A11CB11CC701B6016D5F7F4F8F4F9F4F85
:103CD0009FDE7114F1F08115E1F08150990B4FEFE7
:103CE000489F9001499F300D1124472D4150550B9D
:103CF000240F351F2150310908F48CCF8FE99FE044
:103D00000197F1F700C00000F5CF60E0C801B4D61C
:103D100081CF2496E1E10C946132089508950F93C8
:103D20001F93CF93DF93843008F561111FC0453096
:103D3000E8F4C42FD0E0CC0FDD1F2AE0829FC00D35
:103D4000D11D1124CE0189960E943933082F10E02D
:103D5000102F0027CE018A960E9439339801282B14
:103D6000C901DF91CF911F910F91089580E090E0FC
:103D7000F8CF1F93CF93DF93962F122F632F8430AA
:103D8000B0F4911114C0453090F4C42FD0E0CC0FA2
:103D9000DD1F9AE0899FC00DD11D1124CE018996A7
:103DA0000E945A33612FCE018A960E945A33DF91C6
:103DB000CF911F910895FF920F931F93CF93DF939D
:103DC000F42E843068F5653058F524E0629FE001F8
:103DD000112434E1839FC00DD11D1124CF5ADF4F30
:103DE00081E084279E01280F311D280F311DC90154
:103DF0000E943933082F10E0102F002781E090E057
:103E0000F11002C083E090E08C0F9D1F0E943933B7
:103E10009801282BC901CDB7DEB7E5E00C946D32CF
:103E200080E090E0F8CF0F931F93CF93DF93C62FDE
:103E3000142F022F632F843010F5C53000F524E0D5
:103E4000C29FE001112434E1839FC00DD11D1124D4
:103E5000CF5ADF4F81E084279E01280F311D280FA4
:103E6000311DC9010E945A3381E090E0111102C056
:103E700083E090E0602F8C0F9D1F0E945A33DF91EA
:103E8000CF911F910F910895A0E0B0E0EAE4FFE127
:103E90000C944A326B017C01E80146015701820E05
:103EA000931EA41EB51EC814D904EA04FB0429F409
:103EB000CDB7DEB7ECE00C94663288E2C816D104C8
:103EC000E104F10458F4C60189960E9439338993BC
:103ED0008FEFC81AD80AE80AF80AE5CF80E0F7CFD2
:103EE000A0E0B0E0E6E7FFE10C9444326B017C0116
:103EF00049015A01E80128E2C216D104E104F104A3
:103F000010F588E290E0A0E0B0E08C199D09AE09C0
:103F1000BF0988159905AA05BB05A8F01B0139E260
:103F2000230E311C8091F3029091F402892B81F0D1
:103F300000E010E0C801A0E0B0E0081519051A047F
:103F40001B0408F449C0CDB7DEB7E2E10C9460323F
:103F5000340100E010E0C0FE0DC0CB0188960E9445
:103F60003933988189279827892781159C4789F1BA
:103F700001E010E0D701C601880D991DAA1DBB1DE7
:103F800080FF14C094012150310939012E01420EE5
:103F9000531EC101880D991D0E943933F201908191
:103FA00081159C4719F48FEFF2018083FE01E00F29
:103FB000F11F2FEF0615170508F0BACF9081818108
:103FC00081159C4711F4208321830E5F1F4F329689
:103FD000F1CF8FEF8883CCCF8C0D9D1DAE1DBF1D03
:103FE0008897A105B10548F4FE01E00FF11F60813B
:103FF000C101800F911F0E945A330F5F1F4F9ACF4C
:104000006FE573E080E090E008954F925F926F92C9
:104010007F92AF92BF92CF92DF92EF92FF920F9377
:104020001F93CF93DF936B017C0129013A01580163
:104030008B010F551F4FC0E0D0E0CE01A0E0B0E0F3
:10404000C415D5051604170478F0DF91CF911F91A0
:104050000F91FF90EF90DF90CF90BF90AF907F9047
:104060006F905F904F9008958C0D9D1DAE1DBF1DEC
:104070008F359340A105B10550F4C8018C0F9D1FE9
:104080000E943933F50181935F012196D6CF80E0FC
:10409000F9CF4F925F926F927F92AF92BF92CF9281
:1040A000DF92EF92FF920F931F93CF93DF936B01F9
:1040B0007C0129013A0158018B010F551F4FC0E0C7
:1040C000D0E0CE01A0E0B0E0C415D5051604170479
:1040D00078F0DF91CF911F910F91FF90EF90DF90DB
:1040E000CF90BF90AF907F906F905F904F9008956A
:1040F0008C0D9D1DAE1DBF1D8F359340A105B105D3
:1041000048F4F501EC0FFD1F6081C8018C0F9D1F65
:104110000E945A332196D5CFA0E1B0E0E2E9F0E267
:104120000C944632FE01319680E1DF011D928A95A2
:10413000E9F706E310E09FE5492E93E0592E612C44
:10414000712C21EAA22EB12C4F0173016201B1E161
:104150004B165104610471041CF080E1C82ED12C6F
:10416000A601B501C4010E944B33AC0CBD1C0D2C43
:10417000000CEE08FF084C185D086E087F0801501F
:10418000104019F76096E0E10C946232CF93DF9310
:10419000EB0186319C4719F50E94CA0C9D8191154F
:1041A000A1F08A7A91E0811101C090E090930B0315
:1041B000811549F085E30E943A290E94A60D80E00E
:1041C000DF91CF91089589E2F6CF80910B0381159D
:1041D00021F085E30E945129F0CF89E2FBCF81E0F5
:1041E000EFCFCF93DF93EC01FB018581811509F4BB
:1041F000CBC09E0130572332310508F0ABC08BE2B3
:1042000093E00E943D0EFE01E150F047E232F105DD
:1042100020F4EF52FC4C0C94123280912B038160FD
:1042200080932B0390C080912C03886080932C0393
:104230008AC080912B038260F3CF80912B0384602E
:10424000EFCF80912B038860EBCF80912C038160AE
:10425000EDCF80912C038260E9CF80912B038061A8
:10426000DFCF80912B038062DBCF80912B038064B2
:10427000D7CF0E947A0880912B038068D1CF80919C
:104280002B038C60CDCF80912C038360CFCF8091A6
:104290002B038E7FC5CF80912C03877FC7CF809162
:1042A0002B038D7FBDCF80912B038B7FB9CF809166
:1042B0002B03877FB5CF80912C038E7FB7CF809162
:1042C0002C038D7FB3CF80912B038F7EA9CF80915C
:1042D0002B038F7DA5CF80912B038F7BA1CF0E94D5
:1042E0007A0880912B038F779BCF80912B03837F5C
:1042F00097CF80912C038C7F99CF80912B039927A6
:1043000082FF939590FB82F990FB83F989CF80918E
:104310002C03982F909590FB80F990FB81F986CF24
:1043200090912B03892F8F7B96FF806479CF0E9419
:104330007A0890912B03892F97FB87F9805870CFCB
:1043400081E00E94450E8BE293E00E943F0E0E94A6
:104350007A0880E0DF91CF91089580E0F2CF9091CC
:104360002B03892F8F7E94FF80615ACF90912B036E
:10437000892F8E7F90FF816053CF90912C03892FDE
:10438000877F93FF886052CF81E0E4CF282F35EB01
:104390002303C001112497FF04C080589109892F7D
:1043A000089580589F4FFBCF8091120380FF0DC06E
:1043B0006091200170E0660F771F60387105B0F5DD
:1043C00061157105A9F1862F089581FF07C06091DD
:1043D000200184E0689FB0011124EFCF82FF04C068
:1043E0006091200188E0F6CF909111039115D9F0EA
:1043F00020911F0180912001682F70E0921730F00A
:1044000043E0660F771F4A95E1F7D7CF899FC00138
:10441000112433E0880F991F3A95E1F7622F70E07D
:104420000E94DD31CACF68E070E0CDCF8FE70895FC
:1044300081E008958091120380FF0CC060911C01FF
:1044400070E075956795759567956115710549F1EA
:10445000862F089581FF06C060911C0170E075955C
:104460006795F3CF60911C0182FD0BC09091100302
:104470009115A1F060911B0180911C01961738F0F5
:10448000682F70E06038710500F38FE70895899F09
:10449000C001112470E00E94DD31F4CF61E070E0D2
:1044A000D7CF81E00895E3E3E80FE331A0F5F0E032
:1044B000ED50FC4C0C94123277DF819580931603FB
:1044C000089572DFFBCF70DF819580931503089507
:1044D0006BDFFBCFAFDF809317030895ABDF8195D0
:1044E000FACFA8DF8195809318030895A3DFFBCF4F
:1044F000815D990B21E030E001C0220F8A95EAF737
:1045000080911403822B80931403089580911203E9
:104510008160809312030895809112038260F9CF25
:10452000809112038460F5CF409115038D3C59F4BE
:104530008091160387FF0DC010921603411559F4A0
:104540001092110308C08E3C81F480911603181656
:104550009CF3411581F08091170390911803892BEA
:10456000811159C01092100308958F3C41F447FF08
:10457000F0CF10921503809116038115E0CF803D96
:1045800019F41416B4F3E5CF90911703893D29F47B
:104590001916FCF610921703DCCF8A3D19F497FF29
:1045A000D8CFF8CF909118038B3D29F497FFD1CF46
:1045B00010921803CECF8C3D19F41916CCF3C9CF45
:1045C0009FE2980F983090F4815D990B21E030E0E4
:1045D000B90102C0660F771F8A95E2F7CB0180957B
:1045E00090911403892380931403B3CF8D3D31F44C
:1045F000809112038E7F80931203ABCF8E3D21F406
:10460000809112038D7FF7CF8F3D09F0A2CF80916B
:1046100012038B7FF0CF08957ED720911503309140
:104620001603232B211521F080930E0390930F0383
:104630002091170330911803232B211521F080932B
:104640000C0390930D0383E193E0F5C486E0E3E16E
:10465000F3E0DF011D928A95E9F7109211031092A1
:104660001003109212030895FC01828181110DC084
:10467000838181110AC08481811107C081E0958105
:10468000911101C080E08170089581E0FCCFA6E027
:10469000B0E0EDE4F3E20C94513286E0E3E1F3E0C4
:1046A0009E012F5F3F4FD90101900D928A95E1F74E
:1046B000109215031092160310921703109218030C
:1046C0008B819C81892B8901811581F080910E035A
:1046D00090910F03B1D69C0180911103811599F13E
:1046E000909121019217130608F43AC08D819E81A2
:1046F000892B811589F080910C0390910D039CD634
:104700009C0180911003811509F458C090911D01FE
:104710009217130608F460C0B80183E193E0F1D565
:10472000811104C083E193E09FDF811175DF86E092
:10473000F801A3E1B3E001900D928A95E1F7269686
:10474000E5E00C946D32409122019AE0499FA0016E
:1047500011244217530750F68F5F8093110302C054
:104760008F3FD1F7FB80F11451F01EDE91E01F1452
:104770000CF09FEF899F802D112480931503FC80FE
:10478000F11451F011DE91E01F140CF09FEF899F9E
:10479000802D11248093160380911503811509F44F
:1047A000A5CFF0901603F11409F4A0CFEFDD8093AC
:1047B00015038F2DEBDD8093160398CF40911E01DA
:1047C0009AE0499FA00111244217530708F0A4CF93
:1047D0008F5F8093100302C08F3FD1F7FD80F114EB
:1047E00051F028DE91E01F140CF09FEF899F802D7F
:1047F000112480931703FE80F11451F01BDE91E029
:104800001F140CF09FEF899F802D112480931803B3
:1048100080911703811509F47FCFF0901803F114EC
:1048200009F47ACFB3DD809317038F2DAFDD80932A
:10483000180372CFFC01A081B1818D91B183A08357
:104840000895A0E0B0E0E7E2F4E20C944D32E82FE6
:10485000F0E0EC5BFB4FB490282F2695269526952B
:1048600030E0F901EC51FB4F0491877010E0082E05
:1048700002C0159507950A94E2F701701127F90116
:10488000EC52FB4FE490F12C082E02C0F594E79413
:104890000A94E2F7E0FAEE24FF24E0F8F901EC5381
:1048A000FB4FC491D0E002C0D595C7958A95E2F739
:1048B000C170DD27C62ED12C0115110549F5E11473
:1048C000F10431F086EE0E94BE05C601009771F535
:1048D000B6018B2D0E942F06C601009779F5E114D1
:1048E000F104A1F50115110531F081EE0E940206D7
:1048F000C6010097C9F5CD2B31F08CE20E94450628
:10490000C114D104C9F5CDB7DEB7E9E00C94693222
:1049100081EE0E94BE05C601009789F2EFE9FFE033
:104920003197F1F700C000000197F6CFEFE9FFE003
:104930003197F1F700C000000197C8CFEFE9FFE021
:104940003197F1F700C000000197C7CF86EE0E94B3
:104950000206C601009731F2EFE9FFE03197F1F767
:1049600000C000000197F6CFEFE9FFE03197F1F7C3
:1049700000C000000197BDCF8FE99FE00197F1F7DC
:1049800000C0000091E0C91AD108BACFA0E0B0E0A1
:10499000ECECF4E20C944D328C01D62FF72EE42E81
:1049A0008D2F9F2DF80109958115B9F0813009F0FF
:1049B00060C08D2F9F2DF8010995C82F813091F48B
:1049C0008D2F9F2DF80109950E9445068E2D90E0B0
:1049D000009709F046C0C111E3CFCDB7DEB7E9E0DB
:1049E0000C946932823039F48D2F9F2DF80109958E
:1049F0000E94BE05EBCF833039F48D2F9F2DF80137
:104A000009950E940206E2CF843001F78D2F9F2D79
:104A1000F8010995C82FC12CD12C8AE0B82E2C2F73
:104A20002053330BC9012A30310568F0C114D10479
:104A300069F28FE99FE00197F1F700C0000091E073
:104A4000C91AD108F3CFBC9C9001BD9C300D112434
:104A50006C01C20ED31E8D2F9F2DF8010995C82F12
:104A6000DECFEFE9FFE03197F1F700C000000197DA
:104A7000AFCF6E2DE6DE94CFA2E0B0E0E2E4F5E247
:104A80000C945432462F9A838983BE016F5F7F4F07
:104A90008AE194E27BDF2296E2E00C94703260E0DF
:104AA000EBCF0F931F93CF93DF93C42FD22FFC0133
:104AB00085818115C1F040931B032DD590931A0376
:104AC0008093190380E28C0F883040F4C77081E036
:104AD00001C0880FCA95EAF70E944C06DF91CF917A
:104AE0001F910F91089510911B03141332C08091F0
:104AF000190390911A03A0D4883C910550F5C0E2A7
:104B0000CD0F1D17C1F080E2810F883040F417707F
:104B100081E001C0880F1A95EAF70E945106C8305B
:104B200050F491E08D2F877001C0990F8A95EAF7B4
:104B3000892F0E944C06802F0E944506C83070F6CF
:104B4000D77081E001C0880FDA95EAF70E9451061C
:104B5000C5CF80E28C0F883008F0C0CFC77081E0ED
:104B600001C0880FCA95EAF7F1CF0F93FC01CB0182
:104B7000E851FC47E730F10588F5EA5FFB4C0C94FF
:104B8000123206E221EE41EE6AE17CE78ADF80E044
:104B90000F91089507E225EE45EE6BE17CE7F6CF35
:104BA00006E221EE40EE68E17CE7F0CF07E225EE79
:104BB00044EE69E17CE7EACF06E221EE42EE6CE1E9
:104BC0007CE7E4CF07E225EE46EE6DE17CE7DECF41
:104BD00008E221E045EE6EE17CE7D8CFFB0185815C
:104BE000811110921B0381E0D3CFCF93DF939C01FF
:104BF000FB0127378CE7380739F028373C47C9F0E5
:104C000081E0DF91CF9108958581811571F018D0F1
:104C10000E94EB081BD0D82F16D0C82F11D04D2FD3
:104C20006C2F0E940E0A80E0ECCF0AD00E94F5089B
:104C3000F1CF8581811511F006D0EACF04D0F6CFEF
:104C40008091250108958091240108958091230188
:104C5000089585E290E00E943933863289F486E235
:104C600090E00E94393381110BC087E290E00E94EE
:104C7000393391E08F3C09F090E0892F81700895DD
:104C800080E0FCCFCF93C82F66E2811101C06FEFA7
:104C900085E290E00E945A336FEF6C0F86E290E05D
:104CA0000E945A336FECC11101C06FEF87E290E0B0
:104CB0000E945A33CF910895089588E290E00E94AF
:104CC0003933682F70E080E090E008950895CF9325
:104CD000C62FFCDF6C2F88E290E00E945A33CF9100
:104CE000089580E0CFDF60E070E0CB01F0DF0E944C
:104CF000251D0E94B21D81E0C5CFDEDFDEDFE6DFCD
:104D0000A8DF811101C0EDCF08959C01FB018581D1
:104D1000811551F0A90157574038510530F4822FC1
:104D20000E94B41D80E0089581E008952FEFFC01FA
:104D300020830895CF93DF93EC0188818238C1F0FE
:104D400038F4803871F0813881F0DF91CF91089587
:104D50008338D9F70E94491489830E944C148A83AE
:104D6000F4CF0E944F148983F0CF0E941C14FBCF14
:104D70000E944314F8CFCF93DF93EC0188818238EF
:104D800039F138F4803869F08138B1F0DF91CF9192
:104D900008958338D9F70E944F14482F6A8189817A
:104DA00008C0D9810E944C14C82F0E9449144D2F6D
:104DB0006C2F0E94A015EACF89810E94AF188981CB
:104DC000811103C00E943218E1CF0E94D518DECFB6
:104DD00089810E944614DACF1F93CF93DF93EC01B1
:104DE000162FE8818091F1029091F202892B69F0EF
:104DF000EE3F89F58981833018F08550833058F56E
:104E0000612FCE010E948D1926C0CE010196E4319A
:104E100050F4E11551F0E150E33138F4F0E0E35F94
:104E2000FB4C0C941232EE3F59F3612FCE017EDF22
:104E300012C0198289E08A830EC08981823099F07C
:104E40008330B9F0813089F772D30E9418326A83B7
:104E50007B838C839D83612FCE010E948919DF9112
:104E6000CF911F91089529DF1A821B821C826D83C6
:104E7000F2CF8091F3029091F402892B61F380E0EC
:104E80000E942F12D8CF8981823079F66A817B8186
:104E90008C819D810E9418321ADFDDCF4B816A819F
:104EA00089810E941D1D9827892798279D838C83BF
:104EB000D2CF2C813D813227232732274B816A8133
:104EC00089810E941F1DC7CF0E94251DC4CF53DFBB
:104ED000C2CF30DFC0CF0E940D14BDCF0E94931D02
:104EE0008983B9CF0E94951D9827892798279A838F
:104EF0008983B1CF8B81682F70E08D3108F0ABCF03
:104F000089819A81AE014C5F5F4F98278927982746
:104F10000E94981DA0CF8091F3029091F402892BFA
:104F200009F499CF8B81682F70E08D3108F093CF11
:104F300089819A81AE014C5F5F4F98278927982716
:104F40000E94A51D88CF0E94B21D85CF0E941B1D07
:104F5000C7CF8B81682F70E08D3108F07CCF8981BD
:104F60009A81AE014C5F5F4F9827892798270E944E
:104F7000671D71CF8B81682F70E08D3108F06BCF8A
:104F800089819A81AE014C5F5F4F982789279827C6
:104F90000E94741D60CF8091F3029091F402892BDE
:104FA00009F459CFCE010E9489192FEF81EE94E0C8
:104FB000215080409040E1F700C00000E8D24BCF84
:104FC0009093210380932003089502D2982F81E0CB
:104FD000913009F080E00895E0912003F0912103E1
:104FE000309739F00190F081E02D309711F009955C
:104FF000089580E00895E0912003F0912103309717
:1050000031F00280F381E02D309709F00995089581
:10501000DC01E0912003F0912103309759F0848165
:105020009581892B39F086E08C930480F581E02D01
:10503000CD0109950895DC01E0912003F091210351
:10504000309759F086819781892B39F082E08C93D3
:105050000680F781E02DCD0109950895A3E0B0E029
:10506000E4E3F8E20C9454329C0180911E03909189
:105070001F0382179307B1F030931F0320931E0381
:10508000E0912003F0912103309761F00084F185D5
:10509000E02D309739F083E089833B832A83CE016A
:1050A000019609952396E2E00C947032A3E0B0E0FB
:1050B000ECE5F8E20C9454329C0180911C03909131
:1050C0001D0382179307B1F030931D0320931C0337
:1050D000E0912003F0912103309761F00084F18585
:1050E000E02D309739F084E089833B832A83CE0119
:1050F000019609952396E2E00C947032E09120032A
:10510000F0912103309731F00284F385E02D309740
:1051100009F009950895CF93DF93C0910601D091CE
:105120000701229652DF811581F080912B0387FFC2
:105130000CC0C0910401D091050122969EE180E04F
:10514000915028F4DF91CF91089596E0F8CF2991FE
:105150002115B1F38F5FF4CFCF93C82F811102C017
:1051600080E030C032DF811521F080912B0387FD74
:105170000EC08091060190910701FC0132960896BD
:1051800021912C1709F1E817F907D1F7E9CF8C2FF6
:10519000869586958695C03F18F7E0910401F091B9
:1051A0000501E80FF11D228130E0C77081E090E039
:1051B00002C0880F991FCA95E2F72823392381E09E
:1051C000232B71F2CF91089581E0FCCF9C01FC016B
:1051D00032968FEF90E04191461751F08F3F19F4CE
:1051E000411101C0892F9F5F9630A9F78F3F09F4C5
:1051F0000895280F311D87FD3A95F90162830895BE
:105200009C01FC013296285F3F4F8191861302C0BA
:10521000DF011E92E217F307C1F70895FC01862F04
:10522000869586958695603F60F4E80FF11D67705E
:1052300021E030E001C0220F6A95EAF78281822BDB
:1052400082830895FC01862F869586958695603F1A
:1052500080F4E80FF11D677081E090E09C0102C0CE
:10526000220F331F6A95E2F7B901609582816823A6
:1052700062830895CF93C82FA8DE6C2F811559F053
:1052800080912B0387FF07C0809104019091050155
:10529000C5DFCF910895809106019091070196DFB7
:1052A000F8CFCF93C82F91DE6C2F811559F08091E4
:1052B0002B0387FF07C08091040190910501C2DF95
:1052C000CF910895809106019091070199DFF8CF61
:1052D0007CDE811579F080912B0387FF0BC0E09174
:1052E0000401F091050132968EE1DF011D928A954D
:1052F000E9F70895E0910601F0910701329686E002
:10530000F4CFDC01FB0111969C91119781819813D8
:1053100022C012968C911297811519F092818913EF
:105320001AC013968C911397811519F093818913E4
:1053300012C015968C911597811519F095818913D6
:105340000AC014969C91911521F081E024812913C3
:1053500003C080E001C081E0817008950895FECF10
:1053600008958F5F80932901609126017091270134
:105370008091280190912901F2CF83E08093290147
:105380006091260170912701809128019091290157
:10539000E6CFE7CF089581E080932901609126014F
:1053A000709127018091280190912901D8CFF3CFE6
:1053B000089591E0811101C090E0909328016091DF
:1053C0002601709127018091280190912901C7CF72
:1053D00080912801089580932701609126017091A2
:1053E00027018091280190912901B9CF809127014F
:1053F0000895809326016091260170912701809184
:10540000280190912901ABCF80912601089508953C
:105410000895FECF089508950895F9CF0895FBDF0C
:105420000E948B12F9DF80E00E942F12982F81E0FA
:10543000911101C080E00895CF93DF93EC016BD010
:105440008C1B9D0BDF91CF91089585B7806885BF38
:1054500085B7806885BF08951F921FB61F921124DB
:105460008F939F93AF93BF9380912203811113C0B9
:105470008091480390914903A0914A03B0914B0356
:105480004196A11DB11D8093480390934903A093B9
:105490004A03B0934B03BF91AF919F918F911F909F
:1054A0001FBE1F90189580915003843031F10E94E7
:1054B0003A051092220388E190E020E40FB6F894B8
:1054C000A895809360000FBE2093600083B7817F12
:1054D000846083BF83B7816083BF7894889583B7E6
:1054E0008E7F83BF0FB6F894A89580916000886185
:1054F00080936000109260000FBE08950E947A08A9
:105500000C943E0582E084BD93E095BD9AEF97BD73
:1055100080936E0008952FB7F8948091480390917E
:105520004903A0914A03B0914B032FBF08952FB7B1
:10553000F894609148037091490380914A039091D7
:105540004B032FBF089578941F921FB61F9211240A
:105550008F939F93AF93BF9380914803909149039A
:10556000A0914A03B0914B030196A11DB11D8093F8
:10557000480390934903A0934A03B0934B03BF9110
:10558000AF919F918F911F901FBE1F90189587E735
:1055900097E7909301088093000888E19AE00FB69E
:1055A000F894A895809360000FBE90936000FFCFA1
:1055B00088E19AE00FB6F894A895809360000FBE3A
:1055C00090936000FFCF282FCB01BA013091500398
:1055D0003430D1F42F702093E9002FEF3091E800A0
:1055E00035FD06C035ED3A95F1F700002A95B1F783
:1055F0002091E80025FF08C040E050E0FDD18091F7
:10560000E8008E778093E8000895792F603229F4BE
:1056100040E250E0682F82E0D6CF0895BC0143E01D
:1056200050E084E0D0CFBC0146E050E084E0CBCF36
:10563000BC0140E250E084E0C6CFCF93DF93D82F87
:10564000C92FC6DE48E050E06D2F7C2F81E0BBDF24
:1056500088E0ED2FFC2FA3E2B3E001900D928A9534
:10566000E1F7DF91CF910895A0E2B0E0E9E3FBE23A
:105670001BC7809150038430F9F483E08093E900E4
:105680008091E80082FF18C08091E80090E085FFDB
:1056900008C040E050E060E270E0CE010196F9D130
:1056A00091E08091E8008B778093E800911521F0DC
:1056B00060E2CE01019690DBA096E2E011C78091F6
:1056C0004F03811107C06BD3C2D38091E200846085
:1056D0008093E200089510924F0308955CDE81E00C
:1056E00068CE60914C0381E0611101C080E045CE3D
:1056F0009091500381E0943009F080E060914C0378
:1057000048CE42E061EC81E0C6D242E261EC84E046
:10571000C2D242E261EC82E0BED242E260EC83E0BF
:10572000BAD29091500381E0943009F080E060910A
:105730004C0317CE80915203893081F148F48230B6
:1057400009F496C0833009F457C0813041F00895C0
:105750008A3009F480C08B3009F468C008958091C4
:105760005103813A09F047C08091E800877F809318
:10577000E8008091550390915603892B59F060E021
:1057800080E090E070E0D2D18091E8008B77809348
:10579000E800089568E083E293E0F4CF809151033C
:1057A000813249F580915503909156038D7F892B65
:1057B00011F58091E800877F8093E8008091E800F0
:1057C00082FF15C09091F3008091F200029731F4AE
:1057D0008091F100813011F0863019F48091F10050
:1057E000FADD8091E8008B778093E80088C2809191
:1057F00050038111E3CF089580915103813AD9F785
:105800008091550390915603892BA9F78091E80068
:10581000877F8093E8008091E80080FFFCCFD8DD8F
:105820008093F1008091E8008E77DECF8091510364
:10583000813209F78091550390915603892BD9F64F
:105840008091E800877F8093E80059D280915303CC
:10585000B0DD0C947A0880915103813261F6809119
:10586000E800877F8093E8004AD280915403C1CD3D
:1058700080915103813A09F0BECF8091E800877F83
:105880008093E8008091E80080FFFCCFBDDDC8CFA9
:1058900084B7877F84BF0FB6F894A8958091600085
:1058A000886180936000109260000FBE80E890E0F5
:1058B0000FB6F89480936100909361000FBE77CD8E
:1058C0006ED2C5D2E2EEF0E080818460808378946D
:1058D0002EC58AE291E074CB80915003853029F483
:1058E00080915003853011F009CE0895DCDD97DDFD
:1058F0008115B1F380914E03811591F367D00E9419
:105900007A08EECF08959A014091570350915803B9
:1059100000C0AC01CB01D901252F3327233031053D
:10592000D1F070F42130310509F44BC0223031053B
:1059300069F48BE590E02EE435E02D933C930895D7
:105940002132310509F12232310559F180E090E030
:1059500020E030E0F2CFCA019927423091F0833045
:10596000910538F4EAE2F5E0892B39F4EAE4F5E050
:1059700004C0E4EFF4E0039749F7849190E09F01BD
:10598000DCCFE2E1F5E0F9CF83309105F8F6FC01D8
:10599000EE0FFF1FEA5FFD4F2081318189E090E02B
:1059A000CCCF8330910590F6FC01EE0FFF1FE05045
:1059B000FE4F2081318183509E4FFC01808190E019
:1059C000BCCF82E190E029EA35E0B7CF80E189BD24
:1059D00082E189BD09B400FEFDCF8091D8008F7DA2
:1059E0008093D8008091E00082608093E0008091F5
:1059F000E00081FDFCCF0895AF92BF92CF92DF927D
:105A0000FF920F931F93CF93DF936C01EB018A01F9
:105A100095D1F82E811123C00115110539F0F80137
:105A200080819181C81BD90BC80ED91EA12CB12C25
:105A30002097A9F08091E80085FD21C08091E800C1
:105A40008E778093E80001151105A1F0F80180819F
:105A500091818A0D9B1D9183808385E0F82E8F2D87
:105A6000DF91CF911F910F91FF90DF90CF90BF906A
:105A7000AF90089563D18115E9F2F82EF0CFF601C9
:105A800081916F018093F1002197FFEFAF1ABF0A58
:105A9000CFCFAF92BF92CF92DF92FF920F931F931F
:105AA000CF93DF936C01EB018A0148D1F82E81116D
:105AB00023C00115110539F0F80180819181C81BBF
:105AC000D90BC80ED91EA12CB12C2097A9F080911A
:105AD000E80085FD21C08091E8008B778093E80085
:105AE00001151105A1F0F801808191818A0D9B1D9E
:105AF0009183808385E0F82E8F2DDF91CF911F91C8
:105B00000F91FF90DF90CF90BF90AF90089516D186
:105B10008115E9F2F82EF0CF8091F100F601819322
:105B20006F012197FFEFAF1ABF0ACFCFFC019B0196
:105B300080915703909158038617970718F0672BA9
:105B400061F0C90140E0009771F441110CC08091EF
:105B5000E80082FF35C080E008958091E8008E77EC
:105B60008093E800EECF209150032115A9F1253054
:105B7000A9F12091E80023FD2DC02091E80022FD2D
:105B8000E6CF2091E80020FFDECF3091F300209196
:105B9000F200009719F02830310558F041E0283024
:105BA000310509F040E02091E8002E772093E800CD
:105BB000CACF41914093F10001972F5F3F4FE9CF4A
:105BC00080915003811541F0853041F08091E800CB
:105BD00083FFBDCF81E0089582E0089583E00895BA
:105BE000FC019B01809157039091580386179707FA
:105BF00018F0672B61F0C90140E0009771F4411182
:105C00000CC08091E80082FF36C080E0089580914A
:105C1000E8008E778093E800EECF209150032115A5
:105C2000B1F12530B1F12091E80023FD2EC0209183
:105C3000E80022FDE6CF2091E80020FFDECF309182
:105C4000F3002091F200009719F02830310558F048
:105C500041E02830310509F040E02091E8002E773E
:105C60002093E800CACF44914093F1003196019708
:105C70002F5F3F4FE8CF80915003811541F0853071
:105C800041F08091E80083FFBCCF81E0089582E07D
:105C9000089583E00895982F973028F08F708093AF
:105CA000E90081E008959093E900242F762F50E0D9
:105CB000981731F07091EC002091ED005091F000B8
:105CC00021FD02C09F5FE8CF3091EB003E7F309313
:105CD000EB003091ED003D7F3093ED003091EB0013
:105CE00031603093EB007093EC002093ED00509303
:105CF000F0002091EE0027FDE5CF80E0089580912F
:105D0000510387FF13C08091E80082FF06C0809195
:105D1000E8008B778093E80008958091500381110B
:105D2000F2CF0895809150038115D9F38091E80056
:105D300080FFF8CF8091E8008E77ECCF2091E400CF
:105D40003091E50095E6A9012091EC00822F817049
:105D500020FF06C08091E80080FF06C080E0089523
:105D60002091E80022FD1AC080915003811589F02E
:105D7000853089F08091EB0085FD0FC02091E40013
:105D80003091E50042175307F9F29A95E1F684E065
:105D9000089582E0089583E0089581E0089567D032
:105DA0006ED0E0EEF0E0808181608083E8EDF0E08D
:105DB00080818F77808319BCA7EDB0E08C918E7FB6
:105DC0008C9380818F7E808310924F0308950F9370
:105DD0001F93CF93DF934BD052D0C8EDD0E0888192
:105DE0008F77888388818068888388818F7D888386
:105DF00019BC1092500310924C0310924E03109253
:105E00004D0300EE10E0F80180818B7F8083888154
:105E10008160888342E060E080E03DDFE1EEF0E019
:105E200080818E7F8083E2EEF0E0808181608083DC
:105E3000808188608083F80180818E7F8083888163
:105E400080618883DF91CF911F910F910895E8EDD4
:105E5000F0E080818F7E8083E7EDF0E080818160DB
:105E6000808384E082BF81E080934F03B0CFE8ED70
:105E7000F0E080818E7F80831092E200089510927E
:105E8000DA001092E10008951F920F920FB60F9260
:105E900011242F933F934F935F936F937F938F932F
:105EA0009F93AF93BF93EF93FF938091E10082FFA5
:105EB0000AC08091E20082FF06C08091E1008B7FE2
:105EC0008093E10033D28091DA0080FF18C0809186
:105ED000D80080FF14C08091DA008E7F8093DA00B2
:105EE0008091D90080FF8FC080E189BD82E189BDAA
:105EF00009B400FEFDCF81E080935003E0DB809188
:105F0000E10080FF18C08091E20080FF14C0809102
:105F1000E2008E7F8093E2008091E20080618093B6
:105F2000E2008091D80080628093D80019BC85E09F
:105F300080935003D6DB8091E10084FF28C08091DC
:105F4000E20084FF24C080E189BD82E189BD09B4FB
:105F500000FEFDCF8091D8008F7D8093D800809186
:105F6000E1008F7E8093E1008091E2008F7E80933C
:105F7000E2008091E20081608093E20080914C0316
:105F8000811509F445C084E080935003B1DB809112
:105F9000E10083FF27C08091E20083FF23C080914E
:105FA000E100877F8093E10082E0809350031092AC
:105FB0004C038091E1008E7F8093E1008091E200AC
:105FC0008E7F8093E2008091E20080618093E20006
:105FD00042E060E080E05FDE8091F00088608093C6
:105FE000F0007CDBFF91EF91BF91AF919F918F917A
:105FF0007F916F915F914F913F912F910F900FBEC5
:106000000F901F90189519BC1092500364DB77CF46
:106010008091E30087FF02C083E0B6CF81E0B4CF78
:106020001F920F920FB60F921124EF92FF920F93CF
:106030001F932F933F934F935F936F937F938F9310
:106040009F93AF93BF93CF93EF93FF9309EE10E02D
:10605000F8018081C091EC008F70C795CC27C7955F
:10606000C82B108280EFE82EF12CF7018081877F0A
:10607000808378941FD0F8011082F70180818860B6
:106080008083CF70F801C083FF91EF91CF91BF91D2
:10609000AF919F918F917F916F915F914F913F91C0
:1060A0002F911F910F91FF90EF900F900FBE0F90C7
:1060B0001F901895AAE2B0E0EFE5F0E3F4C181E5A6
:1060C00093E0FC0101962091F100208323E08935C3
:1060D0009207B9F72FDB8091E80083FF37C08091EA
:1060E0005103909152039A3088F5E92FF0E0E05E79
:1060F000FB4C98C1803889F0823841F58091550376
:106100008F70873018F58093E9008091EB0085FB54
:10611000882780F91092E90006C080914E03880F0D
:1061200090914D03892B9091E800977F9093E80020
:106130008093F1001092F1008091E8008E7722C0E8
:10614000811115C080915303813001F18091E800E5
:1061500083FF0AC08091E800877F8093E8008091E8
:10616000EB0080628093EB00AA96E3E0B8C1823036
:1061700069F780915303811581F01092E9008091B5
:10618000E800877F8093E800BADDE0CF81E09330BC
:1061900009F080E080934E03F0CF809155038F701B
:1061A0002FEF280F263090F68093E9002091EB0026
:1061B00020FFE3CF933031F48091EB008062809335
:1061C000EB00DBCF9091EB0090619093EB0021E02E
:1061D00030E0A90102C0440F551F8A95E2F74093B1
:1061E000EA001092EA008091EB008860E8CF81110C
:1061F000ADCF109153031F778091E3008078812BFE
:106200008093E3008091E800877F8093E80077DD4A
:106210008091E80080FFFCCF8091E300806880934C
:10622000E30083E0111101C082E0809350038ECF20
:106230008058823008F08ACF8091530390915403A4
:106240008C3D53E0950791F583E08A838AE2898348
:106250004FB7F894DE01139620E03EE051E2E32FC1
:10626000F0E050935700849120FF03C082958F7017
:106270003F5F8F708A30C0F0895C90E08D939D9372
:106280002F5F243161F74FBF8091E800877F8093B3
:10629000E8006AE270E0CE01019648DC8091E800F7
:1062A0008B778093E80052CF805DE7CF60915503F4
:1062B00070915603AE014F5F5F4F25DBBC01892B08
:1062C00009F444CF8091E800877F8093E8008981BA
:1062D0009A8186DCE3CF803809F038CF8091E800DE
:1062E000877F8093E80080914C038093F10024CF56
:1062F00081112CCF90915303923008F027CF8091D9
:10630000E800877F8093E80090934C03F8DC80914D
:106310004C03811529F084E080935003F2D916CF05
:106320008091E30087FDF7CF81E0F6CF0895CF930A
:1063300080915003811591F08091E900C091EC00AB
:106340008F70C795CC27C795C82B1092E900809114
:10635000E80083FDAFDECF70C093E900CF910895D0
:10636000992778E0880F991F961708F0961B881FC9
:106370007A95C9F78095089587FB082E062687FD34
:10638000819567FD6195ECDF0EF4919507FC819591
:106390000895AA1BBB1B51E107C0AA1FBB1FA6176C
:1063A000B70710F0A61BB70B881F991F5A95A9F7BE
:1063B00080959095BC01CD01089597FB072E16F4AA
:1063C000009406D077FD08D0E4DF07FC05D03EF44A
:1063D000909581959F4F0895709561957F4F089591
:1063E000A1E21A2EAA1BBB1BFD010DC0AA1FBB1FD9
:1063F000EE1FFF1FA217B307E407F50720F0A21B4B
:10640000B30BE40BF50B661F771F881F991F1A94B7
:1064100069F760957095809590959B01AC01BD01E1
:10642000CF010895EE0FFF1F0590F491E02D099420
:10643000692796276927782787277827089505D021
:10644000332312F48A1B9B0B10C0A29FB001B39F91
:10645000C001A39F700D811D1124911DB29F700D6D
:10646000811D1124911D0895F0DFB7FF0895821B4F
:10647000930B0895EADFA59F900DB49F900DA49F04
:10648000800D911D112408952F923F924F925F929B
:106490006F927F928F929F92AF92BF92CF92DF9234
:1064A000EF92FF920F931F93CF93DF93CDB7DEB799
:1064B000CA1BDB0B0FB6F894DEBF0FBECDBF09942D
:1064C0002A88398848885F846E847D848C849B8484
:1064D000AA84B984C884DF80EE80FD800C811B8192
:1064E000AA81B981CE0FD11D0FB6F894DEBF0FBEC1
:1064F000CDBFED010895002E083090F0982F872F22
:10650000762F652F542F432F322F22270850F4CF98
:10651000220F331F441F551F661F771F881F991FA7
:106520000A95B2F7002D089597FD1094002E0830BB
:1065300098F00850232F342F452F562F672F782F90
:10654000892F912DF4CF1594979587957795679519
:1065500057954795379527950A95AAF71124002D49
:1065600008958F929F92AF92BF92CF92DF92EF9257
:10657000FF92CF93DF93EC01688179818A819B81BF
:10658000611571058105910521F464E279ED8BE5D2
:1065900097E02DE133EF41E050E0BAD049015A01D4
:1065A0009B01AC01A7EAB1E465DF6B017C01ACEEB5
:1065B000B4EFA5019401CAD0DC01CB018C0D9D1D67
:1065C000AE1DBF1DB7FF03C00197A109B048888366
:1065D0009983AA83BB839F77DF91CF91FF90EF9040
:1065E000DF90CF90BF90AF909F908F900895B9CFDC
:1065F00080E091E0B6CFA0E0B0E0809300019093FE
:106600000101A0930201B09303010895FB01DC0195
:1066100002C005900D9241505040D8F70895FC01FA
:106620004150504030F001900616D1F73197CF011C
:106630000895882799270895FB01DC0104C08D91F6
:106640000190801921F441505040C8F7881B990BE4
:106650000895FB01DC0102C001900D9241505040B1
:10666000D8F70895DC0101C06D9341505040E0F728
:106670000895F999FECF92BD81BDF89A992780B50A
:106680000895A6E1B0E044E050E034C0A8E1B0E0F5
:1066900042E050E02FC0DC01A40FB51F4150504034
:1066A00040F0CB01840F951F2E9105D041505040F2
:1066B000D8F70895262FF999FECF92BD81BDF89A9B
:1066C000019700B4021639F01FBA20BD0FB6F89436
:1066D000FA9AF99A0FBE08950396272FECDFEADFA6
:1066E000252FE9DF242FE7CF0196272FE4DFE2CF24
:1066F000DC01CB01FC01F999FECF06C0F2BDE1BD82
:10670000F89A319600B40D9241505040B8F7089570
:10671000052E97FB16F400940FD057FD05D060DED0
:1067200007FC02D046F408C050954095309521955D
:106730003F4F4F4F5F4F08959095809570956195AD
:106740007F4F8F4F9F4F0895B7FF94CE93DE821BEC
:10675000930B0895F894FFCF92069206C906C906D6
:1067600035075207BA06BA065607BE07CB07CB074E
:106770001E132113251329132D1331133513391328
:106780003D1341134513A119C119CD19FF191B1A46
:106790003B1A581A6B1AB51ABA1ABD19BD19BD1988
:1067A000C11A4721B6214F2119211D215321212131
:1067B000572163212D21AF213121672135216B2103
:1067C000902139216F2197213F2175217D2125219C
:1067D0005B2129215F21432179218721A021AD213E
:1067E00013214B21BD215C22612263226822782281
:1067F00078227822782278227822782278226A22D7
:106800006E227122762286228C229022D025D625D5
:10681000C125CA25DC25E225E82519271D274327A0
:106820004E2759276427672769276B271527CB270A
:106830006E2772277A278B27A327A627A927BA278F
:106840007A30A030A630A030A630F7301831A6300C
:046850006B317831FF
:10685400010000008C02AC020101020005000505E4
:1068640001191A1B1C1D1E1F202122280850011E5D
:106874000A140103020100000100F6291D2B182B44
:10688400132B0E2B052BE200E900EA00B500B6003D
:10689400B700CD008301CC008A019201940121024A
:1068A400230224022502260227022A02B300B4008E
:1068B4006F0070009F01CB019F02A002E200E9007B
:1068C400EA00B500B600B700CD008301CC008A0110
:1068D40092019401210223022402250226022702A6
:1068E4002A02B300B4006F0070009F01CB019F0225
:1068F400A002F436329734000102020202060606B0
:106904000909090909090F0F0F0F0F0F151515189C
:10691400191919191919191919192324252525259E
:1069240025259F1CA11CAC1CC41CFE06BF5218BA12
:106934004F8A0000FF0100010000FFFF000001007A
:1069440001FF00F5929190C693F6F794664422B63F
:0C6954009306BB05DD056005790599057B
:00000001FF
